 arcsas

 Timestamp is 56d7d157 (Thu Mar 03 11:23:27 2016)

 Preferred load address is 00400000

 Start         Length     Name                   Class
 0001:00000000 00018f70H .text                   CODE
 0001:00018f70 00000010H .text$01                CODE
 0001:00018f80 00007182H .text$s                 CODE
 0002:00000000 00000088H .idata$5                DATA
 0002:00000090 00000428H .rdata                  DATA
 0002:000004b8 00000048H .rdata$debug            DATA
 0002:00000500 00000004H .rdata$sxdata           DATA
 0003:00000000 000004fcH .data                   DATA
 0003:00000500 000001c4H .bss                    DATA
 0004:00000000 0000002eH INIT                    CODE
 0004:00000030 00000028H .idata$2                CODE
 0004:00000058 00000014H .idata$3                CODE
 0004:0000006c 00000088H .idata$4                CODE
 0004:000000f4 00000302H .idata$6                CODE
 0005:00000000 000000c8H .rsrc$01                DATA
 0005:000000d0 00001118H .rsrc$02                DATA

  Address         Publics by Value              Rva+Base       Lib:Object

 0000:00000001       ___safe_se_handler_count   00000001     <absolute>
 0001:00000010       _GetOutstandingIoCnt@4     00401010 f   rxdevice.obj
 0001:000000a0       _NonMSIXInterruptHandler@8 004010a0 f   rxdevice.obj
 0001:00000340       _PMCDpcResponseHandler@16  00401340 f   rxdevice.obj
 0001:00000e80       _PMCInterruptHandler@4     00401e80 f   rxdevice.obj
 0001:00001230       _PMCPushMessageUnitQueueFib@8 00402230 f   rxdevice.obj
 0001:00001950       _RxAccessDeviceRegister@8  00402950 f   rxdevice.obj
 0001:00001b40       _RxCheckAdapterHealth@8    00402b40 f   rxdevice.obj
 0001:00001be0       _RxCheckSyncCommandComplete@8 00402be0 f   rxdevice.obj
 0001:00001d90       _RxDpcInterruptHandler@16  00402d90 f   rxdevice.obj
 0001:00001da0       _RxGetOMRx0@4              00402da0 f   rxdevice.obj
 0001:00001df0       _RxInterruptHandler@4      00402df0 f   rxdevice.obj
 0001:00002030       _RxMapMailBoxFirmwareBase@4 00403030 f   rxdevice.obj
 0001:00002110       _RxNewCommProcessInterrupt@8 00403110 f   rxdevice.obj
 0001:000024c0       _RxNotifyAdapter@12        004034c0 f   rxdevice.obj
 0001:00002570       _RxPullMessageUnitQueueCompletedFib@12 00403570 f   rxdevice.obj
 0001:00002720       _RxPushMessageUnitQueueFib@8 00403720 f   rxdevice.obj
 0001:00002850       _RxSendSynchCommand@48     00403850 f   rxdevice.obj
 0001:000030e0       _RxStartAdapter@8          004040e0 f   rxdevice.obj
 0001:000035b0       _RxWaitForAdapterToBoot@4  004045b0 f   rxdevice.obj
 0001:000036b0       _RxWriteIDR@12             004046b0 f   rxdevice.obj
 0001:00003710       _RxWriteODR@12             00404710 f   rxdevice.obj
 0001:00003790       _SetWaitCount4SendSyncCmd@8 00404790 f   rxdevice.obj
 0001:00003890       _SetWaitCount4StartAdapter@4 00404890 f   rxdevice.obj
 0001:00003900       _SimulateHbaFwTgtFailure@8 00404900 f   rxdevice.obj
 0001:000039c0       _SimulateHbaScsiErros@8    004049c0 f   rxdevice.obj
 0001:00003a50       _RevCheckCompatibility@12  00404a50 f   revision.obj
 0001:00003ae0       _RevGetBuildNumber@0       00404ae0 f   revision.obj
 0001:00003af0       _RevGetExternalRev@0       00404af0 f   revision.obj
 0001:00003b00       _CompareStrings@12         00404b00 f   helpers.obj
 0001:00003b60       _GetDriverParameter@20     00404b60 f   helpers.obj
 0001:00003c60       _LongToAscii@16            00404c60 f   helpers.obj
 0001:00003d10       _MatchRegistryString@8     00404d10 f   helpers.obj
 0001:00003dc0       _ZeroStructure@8           00404dc0 f   helpers.obj
 0001:00003de0       _ArcPrintf                 00404de0 f   arcdebug.obj
 0001:00004040       _GetFwDebugBuffer@8        00405040 f   arcdebug.obj
 0001:00004210       _PutItIntoInternalPrintBuffer@12 00405210 f   arcdebug.obj
 0001:000042d0       _RealSprintf@12            004052d0 f   arcdebug.obj
 0001:00004720       _ChangeIoLimitAndPrintOutstanding@4 00405720 f   timer.obj
 0001:00004810       _CheckFWPulseInCrashDumpMode@4 00405810 f   timer.obj
 0001:000048f0       _CheckingFWAfterPowerStateChange@4 004058f0 f   timer.obj
 0001:00004c80       _ConfigureContainersTimer@4 00405c80 f   timer.obj
 0001:00004df0       _DequeueSortingQTimer@4    00405df0 f   timer.obj
 0001:00004ec0       _MainTimeThread@4          00405ec0 f   timer.obj
 0001:00005110       _RequestAif@4              00406110 f   timer.obj
 0001:00005270       _RequestTimer@16           00406270 f   timer.obj
 0001:00005310       _Reset_IOP_CompletionTimer@4 00406310 f   timer.obj
 0001:000055a0       _RestartAdapterPendingTimer@4 004065a0 f   timer.obj
 0001:00005690       _ReturningKidnappedFibsToOS@4 00406690 f   timer.obj
 0001:00005730       _StopTimer@16              00406730 f   timer.obj
 0001:000057c0       _SynchCommandCompletionTimer@4 004067c0 f   timer.obj
 0001:00005880       _SynchFibCompletionTimer@4 00406880 f   timer.obj
 0001:00005980       _UpdateHBAMappingTable@4   00406980 f   timer.obj
 0001:00005ef0       _VMCloseAllCompletionTimer@4 00406ef0 f   timer.obj
 0001:00006100       _AllocateConsumerProducerCommArea@20 00407100 f   arcinit.obj
 0001:000063b0       _AllocateMessageUnitQueueCommArea@8 004073b0 f   arcinit.obj
 0001:000067c0       _ArcLogEvent@16            004077c0 f   arcinit.obj
 0001:00006850       _ArcLogEventString@24      00407850 f   arcinit.obj
 0001:000068e0       _CheckForVersionMisMatch@4 004078e0 f   arcinit.obj
 0001:00006a10       _CheckMSIxPossibility@4    00407a10 f   arcinit.obj
 0001:00006cc0       _ConfigHBADeviceInit@12    00407cc0 f   arcinit.obj
 0001:00006ef0       _ConfigureContainersRuntime@12 00407ef0 f   arcinit.obj
 0001:00007580       _DriverEntry@8             00408580 f   arcinit.obj
 0001:00007650       _DynamicallyThrottleLunQueueDepth@8 00408650 f   arcinit.obj
 0001:00007880       _FindAdapter@24            00408880 f   arcinit.obj
 0001:000090f0       _GetElapsedSeconds@4       0040a0f0 f   arcinit.obj
 0001:00009180       _GetHBAAdapterProperties@8 0040a180 f   arcinit.obj
 0001:00009230       _GetHbaPhyDevInfo@12       0040a230 f   arcinit.obj
 0001:00009640       _GetHbaPhyDevList@8        0040a640 f   arcinit.obj
 0001:00009a10       _HandleAdapterCommitConfig@4 0040aa10 f   arcinit.obj
 0001:00009ae0       _HandleAdapterConfigIssues@4 0040aae0 f   arcinit.obj
 0001:00009cb0       _HandleAdapterGetConfig@4  0040acb0 f   arcinit.obj
 0001:00009dc0       _HbaDeviceAdd@12           0040adc0 f   arcinit.obj
 0001:00009e90       _HbaDeviceRemove@8         0040ae90 f   arcinit.obj
 0001:00009f40       _HwInitializeAdapter@4     0040af40 f   arcinit.obj
 0001:0000a270       _IOPReset@8                0040b270 f   arcinit.obj
 0001:0000a5e0       _InitializeAdapter@4       0040b5e0 f   arcinit.obj
 0001:0000a6a0       _InitializeConsumerProducerCommRegion@8 0040b6a0 f   arcinit.obj
 0001:0000a8e0       _InitializeConsumerProducerNewAdapter@12 0040b8e0 f   arcinit.obj
 0001:0000a9a0       _InitializeDPCs@4          0040b9a0 f   arcinit.obj
 0001:0000ab40       _InitializeMessageUnitQueueNewAdapter@12 0040bb40 f   arcinit.obj
 0001:0000abe0       _IsAdapterReadyForConfigCommand@4 0040bbe0 f   arcinit.obj
 0001:0000ad20       _LogSystemEvent@28         0040bd20 f   arcinit.obj
 0001:0000ad80       _MapDeviceBase@8           0040bd80 f   arcinit.obj
 0001:0000b1b0       _MatchPciIds@8             0040c1b0 f   arcinit.obj
 0001:0000b330       _ReinitializeAdapterAfterIOPReset@4 0040c330 f   arcinit.obj
 0001:0000b4e0       _ResetAdapter@8            0040c4e0 f   arcinit.obj
 0001:0000bb50       _ReturningLocalOutstandingRequestsToOS@4 0040cb50 f   arcinit.obj
 0001:0000bc50       _ReturningOutstandingSentToFWBeforeIOPResetToOS@4 0040cc50 f   arcinit.obj
 0001:0000bcf0       _SA4ACI2Interface@4        0040ccf0 f   arcinit.obj
 0001:0000bdd0       _SA4CheckMSIx@4            0040cdd0 f   arcinit.obj
 0001:0000be20       _SA4OldCommInterface@4     0040ce20 f   arcinit.obj
 0001:0000be60       _SA4StatusBatching@4       0040ce60 f   arcinit.obj
 0001:0000bf80       _SMCrashDumpModeInitAdapter@8 0040cf80 f   arcinit.obj
 0001:0000c180       _SMNormalModeInitAdapter@8 0040d180 f   arcinit.obj
 0001:0000c3c0       _ScanMapTblForCheck@16     0040d3c0 f   arcinit.obj
 0001:0000c6a0       _ScanMapTblForDeviceAdd@12 0040d6a0 f   arcinit.obj
 0001:0000c870       _ScanMapTblForDeviceRemove@4 0040d870 f   arcinit.obj
 0001:0000c900       _SendEvent2OS@20           0040d900 f   arcinit.obj
 0001:0000cd10       _SendInitStructure@4       0040dd10 f   arcinit.obj
 0001:0000cf00       _SetFwTime@4               0040df00 f   arcinit.obj
 0001:0000cf90       _CompleteQueuedRequest@12  0040df90 f   cmddelivery.obj
 0001:0000d080       _DequeueRawIoReadWriteRequest@12 0040e080 f   cmddelivery.obj
 0001:0000d220       _HandleInterrupt@4         0040e220 f   cmddelivery.obj
 0001:0000d240       _HandleMSIXInterrupt@8     0040e240 f   cmddelivery.obj
 0001:0000d320       _LocalDelay1us@0           0040e320 f   cmddelivery.obj
 0001:0000d320       _Delay1us@0                0040e320 f   arcdebug.obj
 0001:0000d380       _PollSmartHBAFIBCompletion@8 0040e380 f   cmddelivery.obj
 0001:0000d5e0       _PostProcessScsiCommand@16 0040e5e0 f   cmddelivery.obj
 0001:0000d8c0       _ProcessContainerInquiry@16 0040e8c0 f   cmddelivery.obj
 0001:0000de80       _ProcessScsiCommand@12     0040ee80 f   cmddelivery.obj
 0001:0000ea90       _QueuePrintf@12            0040fa90 f   cmddelivery.obj
 0001:0000eb50       _QueueRawIoReadWriteRequest@8 0040fb50 f   cmddelivery.obj
 0001:0000f500       _SendFastIoFib@16          00410500 f   cmddelivery.obj
 0001:0000f530       _SendFib@12                00410530 f   cmddelivery.obj
 0001:0000f7f0       _SendRawIoFib@12           004107f0 f   cmddelivery.obj
 0001:0000fac0       _SendSynchFib@28           00410ac0 f   cmddelivery.obj
 0001:0000fc80       _StartIo@8                 00410c80 f   cmddelivery.obj
 0001:00010630       _AdapterControl@12         00411630 f   cmdproc.obj
 0001:00010cc0       _BuildHBAFib@12            00411cc0 f   cmdproc.obj
 0001:00011160       _BuildHBAIoctlFib@20       00412160 f   cmdproc.obj
 0001:000113b0       _BuildIo@8                 004123b0 f   cmdproc.obj
 0001:00011bd0       _BuildRawIo2ScatterGather4HBAIoctl@16 00412bd0 f   cmdproc.obj
 0001:00011d60       _BuildRawIo2ScatterGather@12 00412d60 f   cmdproc.obj
 0001:00011f10       _BuildRawIoFib@12          00412f10 f   cmdproc.obj
 0001:00012200       _BuildRawIoScatterGather@12 00413200 f   cmdproc.obj
 0001:000123c0       _BuildReadWriteFib@12      004133c0 f   cmdproc.obj
 0001:000126f0       _BuildScatterGather64@16   004136f0 f   cmdproc.obj
 0001:000127a0       _BuildScatterGather@16     004137a0 f   cmdproc.obj
 0001:00012830       _BuildSrbFib@12            00413830 f   cmdproc.obj
 0001:00012a90       _ConvertRawIo2ScatterGather@24 00413a90 f   cmdproc.obj
 0001:00012bb0       _InitializeFib@8           00413bb0 f   cmdproc.obj
 0001:00012be0       _BuildRawScatterGather64@20 00413be0 f   ioctl.obj
 0001:00012c80       _BuildRawScatterGather@20  00413c80 f   ioctl.obj
 0001:00012d10       _CSMIGetControllerConfig@8 00413d10 f   ioctl.obj
 0001:00012e40       _CSMIGetControllerStatus@8 00413e40 f   ioctl.obj
 0001:00012ec0       _CSMIGetDeviceAddress@8    00413ec0 f   ioctl.obj
 0001:00013010       _CSMIGetDriverInfo@8       00414010 f   ioctl.obj
 0001:00013090       _CSMIGetPhyInfo@8          00414090 f   ioctl.obj
 0001:000131f0       _CSMIGetRAIDConfig@8       004141f0 f   ioctl.obj
 0001:00013410       _CSMIGetRAIDInfo@8         00414410 f   ioctl.obj
 0001:00013540       _CSMIGetSATASignature@8    00414540 f   ioctl.obj
 0001:000136a0       _CSMIGetSCSIAddress@8      004146a0 f   ioctl.obj
 0001:000137f0       _CSMISTPPassThru@8         004147f0 f   ioctl.obj
 0001:00013a20       _HandleCSMI@8              00414a20 f   ioctl.obj
 0001:00013b10       _ProcessIoctl@12           00414b10 f   ioctl.obj
 0001:00015f60       _AdapterIsAlive@4          00416f60 f   comm.obj
 0001:00015fa0       _CompleteAllSortingQueue@8 00416fa0 f   comm.obj
 0001:00016020       _CompleteBufferedRequest@12 00417020 f   comm.obj
 0001:000160d0       _CompleteSortingQueueRequest@12 004170d0 f   comm.obj
 0001:00016160       _DeQueueSortingQueue@8     00417160 f   comm.obj
 0001:00016300       _DpcDequeueRawIoReadWriteRequest@16 00417300 f   comm.obj
 0001:00016370       _FreeConsumerProducerAif@8 00417370 f   comm.obj
 0001:00016440       _GetConsumerProducerCompletedFib@12 00417440 f   comm.obj
 0001:000164e0       _GetMessageUnitQueueCompletedFib@12 004174e0 f   comm.obj
 0001:00016500       _GetQueueEntry@16          00417500 f   comm.obj
 0001:00016650       _ProcessAif@8              00417650 f   comm.obj
 0001:00016e00       _ProcessHbaErrors@12       00417e00 f   comm.obj
 0001:00017250       _ProcessNormalFib@20       00418250 f   comm.obj
 0001:00017b30       _QueueSortingQ@8           00418b30 f   comm.obj
 0001:00017d70       _SendConsumerProducerFib@4 00418d70 f   comm.obj
 0001:00017de0       _SendMessageUnitQueueFib@4 00418de0 f   comm.obj
 0001:00017f80       _ServiceHostCommandNormalQueue@4 00418f80 f   comm.obj
 0001:00018020       _ServiceHostResponseNormalQueue@4 00419020 f   comm.obj
 0001:000183d0       _ServiceInternalAifQueue@4 004193d0 f   comm.obj
 0001:00018470       _SubDeQueueSortingQueue@8  00419470 f   comm.obj
 0001:00018540       _TryDeQueueIoList@4        00419540 f   comm.obj
 0001:00018650       _HwScsiWmiExecuteMethod@32 00419650 f   wmi.obj
 0001:000186f0       _HwScsiWmiFunctionControl@20 004196f0 f   wmi.obj
 0001:00018710       _HwScsiWmiQueryDataBlock@32 00419710 f   wmi.obj
 0001:00018730       _HwScsiWmiQueryReginfo@12  00419730 f   wmi.obj
 0001:00018750       _HwScsiWmiSetDataBlock@24  00419750 f   wmi.obj
 0001:00018760       _HwScsiWmiSetDataItem@28   00419760 f   wmi.obj
 0001:00018770       _InitializeWmiInterface@4  00419770 f   wmi.obj
 0001:00018870       _ProcessWmi@8              00419870 f   wmi.obj
 0001:000188d0       _GsDriverEntry@8           004198d0 f   BufferOverflowFastFailK:gs_driverentry.obj
 0001:000188e6       @__security_check_cookie@4 004198e6 f   BufferOverflowFastFailK:secchk.obj
 0001:000188fc       ___report_gsfailure        004198fc f   BufferOverflowFastFailK:gs_report.obj
 0001:00018910       ___report_rangecheckfailure 00419910 f   BufferOverflowFastFailK:gs_report.obj
 0001:0001891a       _memset                    0041991a f   ntoskrnl:ntoskrnl.exe
 0001:00018926       __aulldvrm                 00419926 f   ntoskrnl:ntoskrnl.exe
 0001:00018932       __alldiv                   00419932 f   ntoskrnl:ntoskrnl.exe
 0001:0001893e       __allmul                   0041993e f   ntoskrnl:ntoskrnl.exe
 0001:0001894a       __aulldiv                  0041994a f   ntoskrnl:ntoskrnl.exe
 0001:00018956       __aullshr                  00419956 f   ntoskrnl:ntoskrnl.exe
 0001:00018962       _ScsiPortWmiDispatchFunction@28 00419962 f   scsiwmi:wmilib.obj
 0001:000189de       _ScsiWmipProcessRequest@36 004199de f   scsiwmi:wmilib.obj
 0001:00018d60       _ScsiPortWmiPostProcess@12 00419d60 f   scsiwmi:wmilib.obj
 0001:00018d90       _ScsiWmipPostProcess@24    00419d90 f   scsiwmi:wmilib.obj
 0001:00018efa       _ScsiWmipFindGuid@20       00419efa f   scsiwmi:wmilib.obj
 0001:00018f4a       _ULongAdd@12               00419f4a f i scsiwmi:wmilib.obj
 0001:00018f78       _ForceSEHExceptionHandler@16 00419f78 f   BufferOverflowFastFailK:forceseh.obj
 0001:00018f80       ??_C@_0CJ@KAGJNHLI@OMR?5value?5in?5Check?5Adapter?5Healt@FNODOBFM@ 00419f80     rxdevice.obj
 0001:00018faa       ??_C@_0DE@IHDJGLJF@This?5should?5not?5happen?4?5We?5only?5@FNODOBFM@ 00419faa     rxdevice.obj
 0001:00018fde       ??_C@_0BF@JNCAAJNE@pFibContext?$DNNULL?5?$CB?$CB?6?$AA@FNODOBFM@ 00419fde     rxdevice.obj
 0001:00018ff4       ??_C@_0EM@CCDNION@?$CK?5Start?5a?5timer?5to?5update?5contai@FNODOBFM@ 00419ff4     rxdevice.obj
 0001:00019040       ??_C@_0EF@JHIFCNOI@This?5should?5not?5happen?4?5We?5only?5@FNODOBFM@ 0041a040     rxdevice.obj
 0001:00019086       ??_C@_0DD@DNLJMEID@pFibContext?$DNNULL?5?$CB?$CBline?5?$CFd?5messa@FNODOBFM@ 0041a086     rxdevice.obj
 0001:000190ba       ??_C@_0EG@FJGLAIMH@We?5may?5have?5problem?0?5FW?5is?5idle?0@FNODOBFM@ 0041a0ba     rxdevice.obj
 0001:00019100       ??_C@_0ED@LPIHDLIB@Handle?5IOCTL?5CMD?5with?5vector?50?4?5@FNODOBFM@ 0041a100     rxdevice.obj
 0001:00019144       ??_C@_0BH@CEIDANBI@SHOULD?5NOT?5BE?5HERE?5?$CB?$CB?6?$AA@FNODOBFM@ 0041a144     rxdevice.obj
 0001:0001915c       ??_C@_0DE@MJICMDG@pFibContext?$DNNULL?5?$CB?$CB?5line?5?$CFd?5mess@FNODOBFM@ 0041a15c     rxdevice.obj
 0001:00019190       ??_C@_0ED@DAJFCMJP@?$CK?5Start?5a?5timer?5to?5update?5Contai@FNODOBFM@ 0041a190     rxdevice.obj
 0001:000191d4       ??_C@_0EI@DKKBIMEF@?$CK?5Start?5a?5timer?5to?5update?5contai@FNODOBFM@ 0041a1d4     rxdevice.obj
 0001:0001921c       ??_C@_0BL@OCMKMPMG@PMCPushMessageUnitQueueFib?$AA@FNODOBFM@ 0041a21c     rxdevice.obj
 0001:00019238       ??_C@_0DM@HGFILPIE@SHOULD?5NOT?5BE?5HERE?$CB?5?$CI?$CFs?$CJ?5line?5?$CFd@FNODOBFM@ 0041a238     rxdevice.obj
 0001:00019274       ??_C@_0BE@HCGBMGEE@Vector?5?$CFd?5is?5full?4?6?$AA@FNODOBFM@ 0041a274     rxdevice.obj
 0001:00019288       ??_C@_0CF@MIBCPCJB@SOMETHING?5WRONG?5IN?5LOOPBACK?5CODE@FNODOBFM@ 0041a288     rxdevice.obj
 0001:000192ae       ??_C@_0DE@CKNADHPL@One?5IOTCL?5FIB?5kidnapped?$CB?5FIB_Con@FNODOBFM@ 0041a2ae     rxdevice.obj
 0001:000192e2       ??_C@_0FE@JLKFMCPA@?$CK?5PMCPushMessageUnitQueueFib?3?5Cm@FNODOBFM@ 0041a2e2     rxdevice.obj
 0001:00019336       ??_C@_0FE@JICOMBJP@?$CK?5PMCPushMessageUnitQueueFib?3?5Cm@FNODOBFM@ 0041a336     rxdevice.obj
 0001:0001938a       ??_C@_0EC@LAPIEKPJ@?$CK?5RxSendSynchCommand?3?5mailbox?$FL0?$FN@FNODOBFM@ 0041a38a     rxdevice.obj
 0001:000193cc       ??_C@_0DJ@GJNDHOED@?$CK?5RxSendSynchCommand?3?5mailbox?$FL0?$FN@FNODOBFM@ 0041a3cc     rxdevice.obj
 0001:00019406       ??_C@_0HK@NJDHDGMI@?$CK?5RxSendSynchCommand?3?5There?5is?5a@FNODOBFM@ 0041a406     rxdevice.obj
 0001:00019480       ??_C@_0HB@PLCHFMAA@?$CK?5RxSendSynchCommand?3?5synch?5cmd?3@FNODOBFM@ 0041a480     rxdevice.obj
 0001:000194f2       ??_C@_0EL@HOIBIGPI@?$CK?5RxSendSynchCommand?3?5Got?5respon@FNODOBFM@ 0041a4f2     rxdevice.obj
 0001:0001953e       ??_C@_0EJ@DGPABBLG@?$CK?5RxSendSynchCommand?3?5Should?5NOT@FNODOBFM@ 0041a53e     rxdevice.obj
 0001:00019588       ??_C@_0FA@HKIBFKMH@?$CK?5RxSendSynchCommand?3?5Still?5NO?5r@FNODOBFM@ 0041a588     rxdevice.obj
 0001:000195d8       ??_C@_0KI@HMCHOJIN@?5RxSendSynchCommand?$FLMSIX?5mode?$FN?5f@FNODOBFM@ 0041a5d8     rxdevice.obj
 0001:00019680       ??_C@_0JP@JKCHEOCJ@?5RxSendSynchCommand?$FLMSIX?5mode?$FN?3?5@FNODOBFM@ 0041a680     rxdevice.obj
 0001:00019720       ??_C@_0CN@BCCBJMEA@?5RxSendSynchCommand?5Failed?5?$CFd?0wa@FNODOBFM@ 0041a720     rxdevice.obj
 0001:0001974e       ??_C@_0DB@JEAHJGPL@?$CK?5pDeviceExtension?9?$DOMaxMSIXVecto@FNODOBFM@ 0041a74e     rxdevice.obj
 0001:00019780       ??_C@_0CB@JPABDNKH@?$CK?5Begins?5StatusBatching?0?5Yeaaa?$CB?6@FNODOBFM@ 0041a780     rxdevice.obj
 0001:000197a2       ??_C@_0CF@BPKEMKA@?$CK?5ACI2?5Command?5Delivery?5is?5enabl@FNODOBFM@ 0041a7a2     rxdevice.obj
 0001:000197c8       ??_C@_1DK@JBHFOPMP@?$AAA?$AAd?$AAa?$AAp?$AAt?$AAe?$AAr?$AA?5?$AAC?$AAo?$AAn?$AAf?$AAi?$AAg?$AAu?$AAr?$AAa?$AAt?$AAi?$AAo?$AAn?$AA?5?$AAf?$AAa?$AAi?$AAl?$AAe?$AAd?$AA?$AA@FNODOBFM@ 0041a7c8     rxdevice.obj
 0001:00019802       ??_C@_06CMBKHLEL@Arcsas?$AA@FNODOBFM@ 0041a802     arcdebug.obj
 0001:0001980a       ??_C@_02DKCKIIND@?$CFs?$AA@FNODOBFM@ 0041a80a     arcdebug.obj
 0001:0001980e       ??_C@_0EM@NMLBBIAH@?$CK?5in?5UpdateHBAMappingTable?0?5GetH@FNODOBFM@ 0041a80e     timer.obj
 0001:0001985a       ??_C@_0FA@FCAIGAEL@?$CK?5in?5UpdateHBAMappingTable?0?5GetH@FNODOBFM@ 0041a85a     timer.obj
 0001:000198aa       ??_C@_0GB@FAGGLJPH@?$CK?5First?58?5HBA?5devices?3?5?$CI0x?$CFx?0?$CFd?$CJ@FNODOBFM@ 0041a8aa     timer.obj
 0001:0001990c       ??_C@_0FJ@KOMILNGA@?$CK?5HBA?5mapping?5table?5updated?0?5tim@FNODOBFM@ 0041a90c     timer.obj
 0001:00019966       ??_C@_0GB@HADPCCEF@?$CK?5Start?5a?5timer?5to?5update?5Contai@FNODOBFM@ 0041a966     timer.obj
 0001:000199c8       ??_C@_0CK@JLKEFPAM@entering?5CheckingFWAfterPowerSta@FNODOBFM@ 0041a9c8     timer.obj
 0001:000199f2       ??_C@_0GN@GHJFFNOA@?$CK?5set?5timer?5AGAIN?5in?5CheckingFWA@FNODOBFM@ 0041a9f2     timer.obj
 0001:00019a60       ??_C@_0FK@MIIMDOAD@?$CK?5set?5timer?5AGAIN?5in?5CheckingFWA@FNODOBFM@ 0041aa60     timer.obj
 0001:00019aba       ??_C@_0GB@EDFGCDFC@?$CK?5set?5timer?5AGAIN?5in?5CheckingFWA@FNODOBFM@ 0041aaba     timer.obj
 0001:00019b1c       ??_C@_0N@HAKDCPBM@7?45?40?441063?$AA?$AA@FNODOBFM@ 0041ab1c     timer.obj
 0001:00019b2a       ??_C@_0DO@GCDGNMH@?$CK?5FW?5is?5back?5from?5S3?1S4?4?5StorPor@FNODOBFM@ 0041ab2a     timer.obj
 0001:00019b68       ??_C@_0DM@JABFAEPO@?$CK?5?9?5Reset?5AIFSrb?5to?5NULL?5when?5ba@FNODOBFM@ 0041ab68     timer.obj
 0001:00019ba4       ??_C@_0DN@ELHOMNDM@?$CK?5leaving?5CheckingFWAfterPowerSt@FNODOBFM@ 0041aba4     timer.obj
 0001:00019be2       ??_C@_0DO@OBELKDEH@?$CK?5set?5timer?5AGAIN?5to?5check?5the?5F@FNODOBFM@ 0041abe2     timer.obj
 0001:00019c20       ??_C@_0CI@JPJEKICG@DPC?9Timeout?5may?5happen?5in?5ResetA@FNODOBFM@ 0041ac20     timer.obj
 0001:00019c48       ??_C@_0DH@JNGKJDAE@One?5kidnapped?5FIB?5released?$CB?5FIB_@FNODOBFM@ 0041ac48     timer.obj
 0001:00019c80       ??_C@_0EJ@PCDGPKJP@?$CK?5Driver?5was?5not?5able?5to?5send?5?$CFd@FNODOBFM@ 0041ac80     timer.obj
 0001:00019cca       ??_C@_0DM@PNDEAHOI@?$CK?5Send?5BusChangeDetected?5to?5OS?5i@FNODOBFM@ 0041acca     timer.obj
 0001:00019d06       ??_C@_0FE@KEPMKGLI@?$CK?5Start?5a?5timer?5to?5update?5HBA?5de@FNODOBFM@ 0041ad06     timer.obj
 0001:00019d5a       ??_C@_0EH@FCLGCKBJ@?$CK?5Start?5a?5timer?5to?5update?5HBA?5de@FNODOBFM@ 0041ad5a     timer.obj
 0001:00019da2       ??_C@_0GE@IFJDDHGE@?$CK?5Start?5a?5timer?5to?5update?5Contai@FNODOBFM@ 0041ada2     timer.obj
 0001:00019e06       ??_C@_0DL@DODBJONE@?$CK?5SynchCommandCompletionTimer?3?5S@FNODOBFM@ 0041ae06     timer.obj
 0001:00019e42       ??_C@_0EO@CBNEAKKI@?$CK?5VMCloseAllCompletionTimer?3?5sen@FNODOBFM@ 0041ae42     timer.obj
 0001:00019e90       ??_C@_0FI@MJCPBEAD@?$CK?5VMCloseAllCompletionTimer?3?5wai@FNODOBFM@ 0041ae90     timer.obj
 0001:00019ee8       ??_C@_0DO@ELMMCKMD@?$CK?5VMCloseAllCompletionTimer?3?5SRB@FNODOBFM@ 0041aee8     timer.obj
 0001:00019f26       ??_C@_0EH@BGEEAOIJ@?$CK?5VMCloseAllCompletionTimer?3?5Sho@FNODOBFM@ 0041af26     timer.obj
 0001:00019f6e       ??_C@_0EF@HLMPMNBN@?$CK?5VMCloseAllCompletionTimer?3?5Syn@FNODOBFM@ 0041af6e     timer.obj
 0001:00019fb4       ??_C@_0DH@IBACIAED@?$CK?5SynchFibCompletionTimer?3?5SyncF@FNODOBFM@ 0041afb4     timer.obj
 0001:00019fec       ??_C@_0EC@MICIKMJM@?$CK?5set?5timer?5AGAIN?5to?5check?5the?5F@FNODOBFM@ 0041afec     timer.obj
 0001:0001a02e       ??_C@_0EL@PCHMIFAO@?$CK?5leaving?5Reset_IOP_CompletionTi@FNODOBFM@ 0041b02e     timer.obj
 0001:0001a07a       ??_C@_0CD@MKPFBJDC@leaving?5Reset_IOP_CompletionTime@FNODOBFM@ 0041b07a     timer.obj
 0001:0001a09e       ??_C@_0FK@ODMKKBJL@?$CK?5Start?5a?5timer?5to?5update?5Contai@FNODOBFM@ 0041b09e     timer.obj
 0001:0001a0f8       ??_C@_0FH@GFIHLMMH@?$CK?5Start?5a?5timer?5to?5update?5Contai@FNODOBFM@ 0041b0f8     timer.obj
 0001:0001a150       ??_C@_0DH@KAAGAFOD@?$CK?5leaving?5Reset_IOP_CompletionTi@FNODOBFM@ 0041b150     timer.obj
 0001:0001a188       ??_C@_0DH@DFJOPAAJ@?$CK?5RESET?5IOP?5done?4?5StorPort?5minip@FNODOBFM@ 0041b188     timer.obj
 0001:0001a1c0       ??_C@_0BJ@HIBCALL@ProcessAgeOfSortingQueue?$AA@FNODOBFM@ 0041b1c0     timer.obj
 0001:0001a1da       ??_C@_0DA@GEMOEFPE@Dequeue?5Sorting?5Queue?5failed?5in?5@FNODOBFM@ 0041b1da     timer.obj
 0001:0001a20a       ??_C@_0ID@HFHPGANL@Dequeue?5Sorting?5Queue?5failed?5whe@FNODOBFM@ 0041b20a     timer.obj
 0001:0001a28e       ??_C@_0CL@MJMGCLDD@entering?5AllocateConsumerProduce@FNODOBFM@ 0041b28e     arcinit.obj
 0001:0001a2ba       ??_C@_0DK@IJIOFPFH@leaving?5AllocateConsumerProducer@FNODOBFM@ 0041b2ba     arcinit.obj
 0001:0001a2f4       ??_C@_0CI@FFOEPFMJ@?$CK?5ConsumerProducerCommArea?0?5VAdd@FNODOBFM@ 0041b2f4     arcinit.obj
 0001:0001a31c       ??_C@_0CN@MBHLABKL@?$CK?5Adapter?5got?5an?5invalid?5host?5me@FNODOBFM@ 0041b31c     arcinit.obj
 0001:0001a34a       ??_C@_0DJ@JGKEIEFI@leaving?5AllocateConsumerProducer@FNODOBFM@ 0041b34a     arcinit.obj
 0001:0001a384       ??_C@_0CL@KCDMGIOM@entering?5AllocateMessageUnitQueu@FNODOBFM@ 0041b384     arcinit.obj
 0001:0001a3b0       ??_C@_0FP@JFBPKCDF@?$CK?5AllocateMessageUnitQueueCommAr@FNODOBFM@ 0041b3b0     arcinit.obj
 0001:0001a410       ??_C@_0DM@JMMHKBOC@?$CK?5AllocateMessageUnitQueueCommAr@FNODOBFM@ 0041b410     arcinit.obj
 0001:0001a44c       ??_C@_0DK@BKFHOPDI@leaving?5AllocateMessageUnitQueue@FNODOBFM@ 0041b44c     arcinit.obj
 0001:0001a486       ??_C@_0DA@ICFHAOHF@?$CK?5AllocateMessageUnitQueueCommAr@FNODOBFM@ 0041b486     arcinit.obj
 0001:0001a4b6       ??_C@_0DJ@EGOLHGNF@leaving?5AllocateMessageUnitQueue@FNODOBFM@ 0041b4b6     arcinit.obj
 0001:0001a4f0       ??_C@_0CF@DNFJFJLG@entering?5ConfigureContainersRunt@FNODOBFM@ 0041b4f0     arcinit.obj
 0001:0001a516       ??_C@_0EJ@GFICDCBB@?$CK?5ConfigureContainersRuntime?3?5Re@FNODOBFM@ 0041b516     arcinit.obj
 0001:0001a560       ??_C@_0EF@KJEEMCEN@?$CK?5ConfigureContainersRuntime?3?5Ge@FNODOBFM@ 0041b560     arcinit.obj
 0001:0001a5a6       ??_C@_0EF@JADMGPAN@?$CK?5ConfigureContainersRuntime?3?5Ge@FNODOBFM@ 0041b5a6     arcinit.obj
 0001:0001a5ec       ??_C@_0EM@NKPEDKJ@?$CK?5ConfigureContainersRuntime?3?5no@FNODOBFM@ 0041b5ec     arcinit.obj
 0001:0001a638       ??_C@_0EF@ECHMIPBP@?$CK?5Found?5a?5new?5container?5?9?5tid?3?5?$CF@FNODOBFM@ 0041b638     arcinit.obj
 0001:0001a67e       ??_C@_0DK@FCJKMAGD@ConfigureContainersRuntime?3?5UID?5@FNODOBFM@ 0041b67e     arcinit.obj
 0001:0001a6b8       ??_C@_0DK@PHPDGAOG@?$CK?5ConfigureContainersRuntime?3?5di@FNODOBFM@ 0041b6b8     arcinit.obj
 0001:0001a6f2       ??_C@_0GG@BFFFADFC@?$CK?5ConfigureContainersRuntime?3?5Fa@FNODOBFM@ 0041b6f2     arcinit.obj
 0001:0001a758       ??_C@_0EA@JBBLNOGE@?$CK?5ConfigureContainersRuntime?3?5RA@FNODOBFM@ 0041b758     arcinit.obj
 0001:0001a798       ??_C@_0FJ@MOJFHLFO@?$CK?5ConfigureContainersRuntime?3?5Di@FNODOBFM@ 0041b798     arcinit.obj
 0001:0001a7f2       ??_C@_0CO@FOBCLEMJ@?$CK?5ConfigureContainersRuntime?3?5di@FNODOBFM@ 0041b7f2     arcinit.obj
 0001:0001a820       ??_C@_0DO@KMBICFHC@?$CK?5ConfigureContainersRuntime?3?5Sy@FNODOBFM@ 0041b820     arcinit.obj
 0001:0001a85e       ??_C@_0DB@JMFIFBDA@leaving?5ConfigureContainersRunti@FNODOBFM@ 0041b85e     arcinit.obj
 0001:0001a890       ??_C@_0CC@KOGKIGDL@entering?5CheckForVersionMisMatch@FNODOBFM@ 0041b890     arcinit.obj
 0001:0001a8b2       ??_C@_0CB@BOFDNAKM@This?5is?5a?5code?5stream?5identifier@FNODOBFM@ 0041b8b2     arcinit.obj
 0001:0001a8d4       ??_C@_0DF@MNNMPGOO@?$CK?5Version?5Mismatch?3?5Bios?3?$CFd?0?5Fir@FNODOBFM@ 0041b8d4     arcinit.obj
 0001:0001a90a       ??_C@_1CE@PCDJGPON@?$AAB?$AAa?$AAd?$AA?5?$AAV?$AAe?$AAr?$AAs?$AAi?$AAo?$AAn?$AA?5?$AAM?$AAa?$AAt?$AAc?$AAh?$AA?$AA@FNODOBFM@ 0041b90a     arcinit.obj
 0001:0001a92e       ??_C@_0EC@DEDLMEPI@leving?5CheckForVersionMisMatch?5w@FNODOBFM@ 0041b92e     arcinit.obj
 0001:0001a970       ??_C@_0BN@GKEKJNDP@?$CFs?5Driver?5entry?5rtnval?5?$DN?5?$CFx?6?$AA@FNODOBFM@ 0041b970     arcinit.obj
 0001:0001a98e       ??_C@_0DD@FIIKPLIC@?$CFs?3?5Driver?5FindAdapter?5?9?5invalid@FNODOBFM@ 0041b98e     arcinit.obj
 0001:0001a9c2       ??_C@_0BG@INJAEJHE@entering?5FindAdapter?6?$AA@FNODOBFM@ 0041b9c2     arcinit.obj
 0001:0001a9d8       ??_C@_0FD@NLKPIIHJ@?$CK?5This?5is?5WS03?5R2?0?5Vista?5or?5Long@FNODOBFM@ 0041b9d8     arcinit.obj
 0001:0001aa2c       ??_C@_0FF@EIPBDAPC@?$CK?$CK?$CK?$CK?$CK?5Size?5of?5PORT_CONFIGURATION@FNODOBFM@ 0041ba2c     arcinit.obj
 0001:0001aa82       ??_C@_0EF@MDPAOPOH@?$CK?5HwScsiFindAdapter?3?5DeviceExten@FNODOBFM@ 0041ba82     arcinit.obj
 0001:0001aac8       ??_C@_0CD@BBBDOKPE@?$CK?5Returned?5PCI?5bus?5data?5length?$DN?$CF@FNODOBFM@ 0041bac8     arcinit.obj
 0001:0001aaec       ??_C@_0BB@ELNGMCEN@BreakPointHelper?$AA@FNODOBFM@ 0041baec     arcinit.obj
 0001:0001aafe       ??_C@_0BN@NMODDHNP@?$CK?53?5seconds?5waiting?5is?5done?6?$AA@FNODOBFM@ 0041bafe     arcinit.obj
 0001:0001ab1c       ??_C@_0DD@OAOECDIB@leaving?5FindAdapter?5?9?5StorPortGe@FNODOBFM@ 0041bb1c     arcinit.obj
 0001:0001ab50       ??_C@_0DF@ODNFGMFG@?$CK?5leaving?5FindAdapter?5?9?5StorPort@FNODOBFM@ 0041bb50     arcinit.obj
 0001:0001ab86       ??_C@_0BN@FJDEMAMC@?$CK?50x40?5PCI?5Bus?5Data?5read?5in?6?$AA@FNODOBFM@ 0041bb86     arcinit.obj
 0001:0001aba4       ??_C@_0BN@INBKDNHG@?$CK?50xFF?5PCI?5Bus?5Data?5read?5in?6?$AA@FNODOBFM@ 0041bba4     arcinit.obj
 0001:0001abc2       ??_C@_0DB@DAIGEFPJ@?$CK?5No?5Support?5on?5Capabilties?5list@FNODOBFM@ 0041bbc2     arcinit.obj
 0001:0001abf4       ??_C@_0BM@KCLFMKNE@?$CK?5Capability_offset?5?$DN?50x?$CFx?5?$AA@FNODOBFM@ 0041bbf4     arcinit.obj
 0001:0001ac10       ??_C@_0BJ@KNABCMMM@?5?9?9?$DOcapabilty_id?5?$DN?50x?$CFx?6?$AA@FNODOBFM@ 0041bc10     arcinit.obj
 0001:0001ac2a       ??_C@_0BK@JIIOJNIO@?$CK?5Message_control?5?$DN?50x?$CFx?6?$AA@FNODOBFM@ 0041bc2a     arcinit.obj
 0001:0001ac44       ??_C@_0BF@HNFCBKLM@?$CK?5HW?5supports?5MSI?9X?6?$AA@FNODOBFM@ 0041bc44     arcinit.obj
 0001:0001ac5a       ??_C@_0DI@MNEPEDIK@?$CK?5StorPortGetActiveGroupCount?5ha@FNODOBFM@ 0041bc5a     arcinit.obj
 0001:0001ac92       ??_C@_0ED@JJDFFHPI@?$CK?5StorPortGetActiveGroupCount?5re@FNODOBFM@ 0041bc92     arcinit.obj
 0001:0001acd6       ??_C@_0DF@EDOFIEGL@?$CK?5StorPortGetGroupAffinity?5has?5n@FNODOBFM@ 0041bcd6     arcinit.obj
 0001:0001ad0c       ??_C@_0HE@CADMEBCK@?$CK?5StorPortGetGroupAffinity?5retur@FNODOBFM@ 0041bd0c     arcinit.obj
 0001:0001ad80       ??_C@_0EI@OFPHCHHN@?$CK?5StorPortGetGroupAffinity?5retur@FNODOBFM@ 0041bd80     arcinit.obj
 0001:0001adc8       ??_C@_0EO@MADFJJKE@?$CK?5StorPortGetGroupAffinity?5retur@FNODOBFM@ 0041bdc8     arcinit.obj
 0001:0001ae16       ??_C@_0DO@FMAFBNDE@?$CK?5StorPortGetCurrentProcessorNum@FNODOBFM@ 0041be16     arcinit.obj
 0001:0001ae54       ??_C@_0FJ@MEGLAFKH@?$CK?5StorPortGetCurrentProcessorNum@FNODOBFM@ 0041be54     arcinit.obj
 0001:0001aeae       ??_C@_0FB@CBENABKH@?$CK?5StorPortGetCurrentProcessorNum@FNODOBFM@ 0041beae     arcinit.obj
 0001:0001af00       ??_C@_0DH@HFNKHLG@?$CK?5StorPortGetActiveNodeCount?5has@FNODOBFM@ 0041bf00     arcinit.obj
 0001:0001af38       ??_C@_0EB@INKBMOFB@?$CK?5StorPortGetActiveNodeCount?5ret@FNODOBFM@ 0041bf38     arcinit.obj
 0001:0001af7a       ??_C@_0EK@DOGGEIOO@?$CK?5StorPortGetActiveNodeCount?5ret@FNODOBFM@ 0041bf7a     arcinit.obj
 0001:0001afc4       ??_C@_0EB@LCBJMNLA@?$CK?5StorPortGetGroupAffinity?5retur@FNODOBFM@ 0041bfc4     arcinit.obj
 0001:0001b006       ??_C@_0DJ@FDFDEBND@?$CK?5StorPortGetHighestNodeNumber?5h@FNODOBFM@ 0041c006     arcinit.obj
 0001:0001b040       ??_C@_0EL@PIGODLHL@?$CK?5StorPortGetHighestNodeNumber?5r@FNODOBFM@ 0041c040     arcinit.obj
 0001:0001b08c       ??_C@_0EM@HBPALBEJ@?$CK?5StorPortGetHighestNodeNumber?5r@FNODOBFM@ 0041c08c     arcinit.obj
 0001:0001b0d8       ??_C@_04GGLOKIEE@dump?$AA@FNODOBFM@ 0041c0d8     arcinit.obj
 0001:0001b0de       ??_C@_05FDLGEGEK@ntldr?$AA@FNODOBFM@ 0041c0de     arcinit.obj
 0001:0001b0e4       ??_C@_05PMICOLGA@hiber?$AA@FNODOBFM@ 0041c0e4     arcinit.obj
 0001:0001b0ea       ??_C@_0CD@JEMNEMMP@?$CK?$CK?$CK?$CK?5dump?5?$HM?5ntldr?5?$HM?5hiber?5is?5TRU@FNODOBFM@ 0041c0ea     arcinit.obj
 0001:0001b10e       ??_C@_0BK@NELCFLHO@?$CK?5Switching?5to?5INTx?5mode?6?$AA@FNODOBFM@ 0041c10e     arcinit.obj
 0001:0001b128       ??_C@_09IPELKJIO@BLEDCheck?$AA@FNODOBFM@ 0041c128     arcinit.obj
 0001:0001b132       ??_C@_0L@NIPCGJOG@DPCAllowed?$AA@FNODOBFM@ 0041c132     arcinit.obj
 0001:0001b13e       ??_C@_09CHINNNMJ@CSMI?$DNNone?$AA@FNODOBFM@ 0041c13e     arcinit.obj
 0001:0001b148       ??_C@_0BA@BKKNJKOP@CSMI?$DNRestricted?$AA@FNODOBFM@ 0041c148     arcinit.obj
 0001:0001b158       ??_C@_09PKBPEONE@CSMI?$DNFull?$AA@FNODOBFM@ 0041c158     arcinit.obj
 0001:0001b162       ??_C@_0CJ@JHBMKCEI@leaving?5FindAdapter?5?9?5PCI?5Id?5not@FNODOBFM@ 0041c162     arcinit.obj
 0001:0001b18c       ??_C@_0CL@HDBMPJMP@?$CK?5leaving?5FindAdapter?5?9?5PCI?5Id?5n@FNODOBFM@ 0041c18c     arcinit.obj
 0001:0001b1b8       ??_C@_0CH@LNPKNDMP@Rx?3?5BAR0?5Range?50x?$CFlx?5MappedSize?5@FNODOBFM@ 0041c1b8     arcinit.obj
 0001:0001b1e0       ??_C@_0DF@OFCBAPFL@leaving?5FindAdapter?5?9?5fail?5mappi@FNODOBFM@ 0041c1e0     arcinit.obj
 0001:0001b216       ??_C@_0DH@MNDLADLD@?$CK?5leaving?5FindAdapter?5?9?5fail?5map@FNODOBFM@ 0041c216     arcinit.obj
 0001:0001b24e       ??_C@_0DC@NODBFDAD@leaving?5FindAdapter?5?9?5illegal?5FW@FNODOBFM@ 0041c24e     arcinit.obj
 0001:0001b280       ??_C@_0EH@FLDBENFC@?$CK?5leaving?5FindAdapter?5?9?5illegal?5@FNODOBFM@ 0041c280     arcinit.obj
 0001:0001b2c8       ??_C@_0CD@NJEIKDOH@?$CK?5New?5outstanding?5number?5chose?3?$CF@FNODOBFM@ 0041c2c8     arcinit.obj
 0001:0001b2ec       ??_C@_0CD@CCLGIJ@?$CK?5Old?5outstanding?5number?5chose?3?$CF@FNODOBFM@ 0041c2ec     arcinit.obj
 0001:0001b310       ??_C@_0N@OEGLNJCG@ioctlbufsize?$AA@FNODOBFM@ 0041c310     arcinit.obj
 0001:0001b31e       ??_C@_0CI@LFOBEGIG@?$CK?5This?5is?564?9bit?5Vista?5or?5Longho@FNODOBFM@ 0041c31e     arcinit.obj
 0001:0001b346       ??_C@_0DB@NLEKMFMO@?$CK?5This?5is?532?9bit?5WS03?5R2?0?5Vista?5@FNODOBFM@ 0041c346     arcinit.obj
 0001:0001b378       ??_C@_0CA@DJAEOOFI@?$CK?5This?5is?564?9bit?5WS03?5SP1?5?4?4?4?5?6?$AA@FNODOBFM@ 0041c378     arcinit.obj
 0001:0001b398       ??_C@_0CA@IELABMFO@?$CK?5This?5is?532?9bit?5WS03?5SP1?5?4?4?4?5?6?$AA@FNODOBFM@ 0041c398     arcinit.obj
 0001:0001b3b8       ??_C@_0CA@MNGBKCLD@?$CK?5This?5is?532?9bit?5WS03?5RTM?5?4?4?4?5?6?$AA@FNODOBFM@ 0041c3b8     arcinit.obj
 0001:0001b3d8       ??_C@_0BL@FPDNGGII@?$CK?5Adapter?5is?5in?5poll?5mode?6?$AA@FNODOBFM@ 0041c3d8     arcinit.obj
 0001:0001b3f4       ??_C@_0CO@NGAJFGIM@?$CK?5pDeviceExtension?9?$DONewCommInter@FNODOBFM@ 0041c3f4     arcinit.obj
 0001:0001b422       ??_C@_0CE@MCFGELJ@?$CK?5pDeviceExtension?9?$DOVendorId?3?50x@FNODOBFM@ 0041c422     arcinit.obj
 0001:0001b446       ??_C@_0CE@PNKCKBKJ@?$CK?5pDeviceExtension?9?$DODeviceId?3?50x@FNODOBFM@ 0041c446     arcinit.obj
 0001:0001b46a       ??_C@_0CH@NNKEKBEL@?$CK?5pDeviceExtension?9?$DOSubVendorId?3@FNODOBFM@ 0041c46a     arcinit.obj
 0001:0001b492       ??_C@_0CH@BEBMHIHH@?$CK?5pDeviceExtension?9?$DOSubSystemId?3@FNODOBFM@ 0041c492     arcinit.obj
 0001:0001b4ba       ??_C@_0CO@NHBGNFPE@?$CK?5Driver?5got?564?5bit?5FIB?5support?5@FNODOBFM@ 0041c4ba     arcinit.obj
 0001:0001b4e8       ??_C@_0CB@ELGCJIGA@?$CK?5Uncached?5Memory?5address?3?50x?$CFp?6@FNODOBFM@ 0041c4e8     arcinit.obj
 0001:0001b50a       ??_C@_0CH@CKCEEBMD@?$CK?5Uncached?5Memory?5allocated?3?50x?$CF@FNODOBFM@ 0041c50a     arcinit.obj
 0001:0001b532       ??_C@_0DK@INJPNBCP@?$CK?5MailBox?51?3?$CFx?0?5MailBox?52?3?$CFx?0?5Ma@FNODOBFM@ 0041c532     arcinit.obj
 0001:0001b56c       ??_C@_0DB@DBAPOAM@?$CK?5pDeviceExtension?9?$DOMaxOutstandi@FNODOBFM@ 0041c56c     arcinit.obj
 0001:0001b59e       ??_C@_0DF@CKKIGFIG@?$CK?5pDeviceExtension?9?$DOMaxMSIXVecto@FNODOBFM@ 0041c59e     arcinit.obj
 0001:0001b5d4       ??_C@_0EC@KMMHNEKL@?$CK?5ConfigInfo?9?$DOHwMSInterruptRouti@FNODOBFM@ 0041c5d4     arcinit.obj
 0001:0001b616       ??_C@_0BH@CDLDBOJF@?$CK?5SrbExtensionSize?3?$CFx?6?$AA@FNODOBFM@ 0041c616     arcinit.obj
 0001:0001b62e       ??_C@_0EK@GNODIBNL@?$CK?5MiniARC?5Interface?5?9?5?5CommandSi@FNODOBFM@ 0041c62e     arcinit.obj
 0001:0001b678       ??_C@_0EL@HJMLPDNI@?$CK?5New?5Comm?5Interface?5?9?5?5CommandS@FNODOBFM@ 0041c678     arcinit.obj
 0001:0001b6c4       ??_C@_0CM@NKHNJDEG@leaving?5FindAdapter?5?9?5fail?5initi@FNODOBFM@ 0041c6c4     arcinit.obj
 0001:0001b6f0       ??_C@_0CO@GHEIBKDI@?$CK?5leaving?5FindAdapter?5?9?5fail?5ini@FNODOBFM@ 0041c6f0     arcinit.obj
 0001:0001b71e       ??_C@_1EA@GNKDGDHK@?$AAA?$AAd?$AAa?$AAp?$AAt?$AAe?$AAr?$AA?5?$AAg?$AAo?$AAt?$AA?5?$AAi?$AAn?$AAv?$AAa?$AAl?$AAi?$AAd?$AA?5?$AAh?$AAo?$AAs?$AAt?$AA?5?$AAw?$AAi?$AAn?$AAd?$AAo?$AAw?$AA?$AA@FNODOBFM@ 0041c71e     arcinit.obj
 0001:0001b75e       ??_C@_1EI@NELDFHEH@?$AAA?$AAd?$AAa?$AAp?$AAt?$AAe?$AAr?$AA?5?$AAd?$AAo?$AAe?$AAs?$AA?5?$AAn?$AAo?$AAt?$AA?5?$AAs?$AAu?$AAp?$AAp?$AAo?$AAr?$AAt?$AA?5?$AA4?$AAG?$AAB?$AA?5?$AAw?$AAi?$AAn@FNODOBFM@ 0041c75e     arcinit.obj
 0001:0001b7a6       ??_C@_0DC@BFHJHJOO@?$CK?5fail?5SynFibCT_SET_MINIARC_HOST@FNODOBFM@ 0041c7a6     arcinit.obj
 0001:0001b7d8       ??_C@_0CE@IADADNNA@?$CK?5Use?5MU?5Register?5for?5IOP_Reset?4@FNODOBFM@ 0041c7d8     arcinit.obj
 0001:0001b7fc       ??_C@_0CJ@LHHNJCHI@?$CK?5Use?5inbound?5doorbell?5for?5IOP_R@FNODOBFM@ 0041c7fc     arcinit.obj
 0001:0001b826       ??_C@_0DI@LGINDMLA@?$CK?5ERROR?3?5FW?5does?5not?5provide?5whi@FNODOBFM@ 0041c826     arcinit.obj
 0001:0001b85e       ??_C@_0BP@DJKPJIGJ@?$CK?5Ignore_IOP_Reset?5is?5set?5?4?4?4?6?$AA@FNODOBFM@ 0041c85e     arcinit.obj
 0001:0001b87e       ??_C@_0CK@LEDHDPPJ@?$CK?5Disk?5Power?5Management?5is?5suppo@FNODOBFM@ 0041c87e     arcinit.obj
 0001:0001b8a8       ??_C@_0CJ@PJOACPGJ@?$CK?5This?5firmware?5supports?5fast?5JB@FNODOBFM@ 0041c8a8     arcinit.obj
 0001:0001b8d2       ??_C@_0DB@HEHLEMPI@?$CK?5Controller?5Firmware?5supports?5S@FNODOBFM@ 0041c8d2     arcinit.obj
 0001:0001b904       ??_C@_0CI@CJPAOACI@?$CK?5Controller?5Firmware?5supports?52@FNODOBFM@ 0041c904     arcinit.obj
 0001:0001b92c       ??_C@_0DA@OBMGONKI@?$CK?5Driver?5got?5SUPPORTED_NATIVE_HB@FNODOBFM@ 0041c92c     arcinit.obj
 0001:0001b95c       ??_C@_0DI@GIKAIFLA@?$CK?5Driver?5did?5not?5get?5SUPPORTED_N@FNODOBFM@ 0041c95c     arcinit.obj
 0001:0001b994       ??_C@_0BH@LMHJIEKF@?$CK?5ExposeNonDASD?5is?5?$CFx?6?$AA@FNODOBFM@ 0041c994     arcinit.obj
 0001:0001b9ac       ??_C@_0BB@JIKBMNNG@QueueDepthPerLun?$AA@FNODOBFM@ 0041c9ac     arcinit.obj
 0001:0001b9be       ??_C@_0N@GDDJMKFE@PauseIOLimit?$AA@FNODOBFM@ 0041c9be     arcinit.obj
 0001:0001b9cc       ??_C@_0O@LIIBGGCF@ResumeIOLimit?$AA@FNODOBFM@ 0041c9cc     arcinit.obj
 0001:0001b9da       ??_C@_0O@OKMDGJBG@ConvertSGList?$AA@FNODOBFM@ 0041c9da     arcinit.obj
 0001:0001b9e8       ??_C@_0BE@IIJOOEPG@QueueStartThreshold?$AA@FNODOBFM@ 0041c9e8     arcinit.obj
 0001:0001b9fc       ??_C@_0BD@CEDPKLI@QueueDumpThreshold?$AA@FNODOBFM@ 0041c9fc     arcinit.obj
 0001:0001ba10       ??_C@_0BA@NLIGFJMK@MaxIoSizeQueued?$AA@FNODOBFM@ 0041ca10     arcinit.obj
 0001:0001ba20       ??_C@_0N@MLHJOFDC@QueueAllowed?$AA@FNODOBFM@ 0041ca20     arcinit.obj
 0001:0001ba2e       ??_C@_0BC@IEBJFOIJ@FlushSizeInBlocks?$AA@FNODOBFM@ 0041ca2e     arcinit.obj
 0001:0001ba40       ??_C@_0EA@OJJGPBKL@leaving?5FindAdapter?5?9?5fail?5Handl@FNODOBFM@ 0041ca40     arcinit.obj
 0001:0001ba80       ??_C@_0EC@HNCBOCML@?$CK?5leaving?5FindAdapter?5?9?5fail?5Han@FNODOBFM@ 0041ca80     arcinit.obj
 0001:0001bac2       ??_C@_09NBOIBGGK@EnableWMI?$AA@FNODOBFM@ 0041cac2     arcinit.obj
 0001:0001bacc       ??_C@_0DH@OIMAJCMK@?$CK?5?9?5Driver?5version?5?$CFs?0?5adapter?5n@FNODOBFM@ 0041cacc     arcinit.obj
 0001:0001bb04       ??_C@_0DF@NGIHOECA@?$CK?5?9?5Size?5of?5HwDevExt?$DN0x?$CFx?4?5Size?5@FNODOBFM@ 0041cb04     arcinit.obj
 0001:0001bb3a       ??_C@_0BG@JAEBOKND@?$CK?5?9?5Done?5FindAdapter?6?$AA@FNODOBFM@ 0041cb3a     arcinit.obj
 0001:0001bb50       ??_C@_0FF@LMEIGAGF@?$CK?5?9?5ConfigInfo?9?$DOMaximumTransferL@FNODOBFM@ 0041cb50     arcinit.obj
 0001:0001bba6       ??_C@_0CG@GOHAMHPA@leaving?5FindAdapter?5?9?5adapter?5fo@FNODOBFM@ 0041cba6     arcinit.obj
 0001:0001bbcc       ??_C@_0BN@DGMFEGDN@entering?5GetElapsedSeconds?5?6?$AA@FNODOBFM@ 0041cbcc     arcinit.obj
 0001:0001bbea       ??_C@_0DD@GOLHMOHG@leaving?5GetElapsedSeconds?5?9?5seco@FNODOBFM@ 0041cbea     arcinit.obj
 0001:0001bc1e       ??_C@_0CJ@KCPJKGH@entering?5IsAdapterReadyForConfig@FNODOBFM@ 0041cc1e     arcinit.obj
 0001:0001bc48       ??_C@_0DB@PNDBFHEI@IsAdapterReadyForConfigCommand?3?5@FNODOBFM@ 0041cc48     arcinit.obj
 0001:0001bc7a       ??_C@_0CH@PFKKGKLP@IsAdapterReadyForConfigCommand?3?5@FNODOBFM@ 0041cc7a     arcinit.obj
 0001:0001bca2       ??_C@_0DJ@FMKIDFML@?$CK?5leaving?5IsAdapterReadyForConfi@FNODOBFM@ 0041cca2     arcinit.obj
 0001:0001bcdc       ??_C@_0CI@LLJGECEO@leaving?5IsAdapterReadyForConfigC@FNODOBFM@ 0041ccdc     arcinit.obj
 0001:0001bd04       ??_C@_0BD@LJONEFCN@entering?5IOPReset?6?$AA@FNODOBFM@ 0041cd04     arcinit.obj
 0001:0001bd18       ??_C@_0EN@CPGMGMBD@?$CK?$CK?5Fail?5to?5iopreset?5the?5adapter?5@FNODOBFM@ 0041cd18     arcinit.obj
 0001:0001bd66       ??_C@_1CG@OOCCJMGE@?$AAI?$AAO?$AAP?$AA?5?$AAR?$AAE?$AAS?$AAE?$AAT?$AA?5?$AAd?$AAi?$AAs?$AAa?$AAb?$AAl?$AAe?$AAd?$AA?$AA@FNODOBFM@ 0041cd66     arcinit.obj
 0001:0001bd8c       ??_C@_1CC@HLNFBNCO@?$AAI?$AAO?$AAP?$AA?5?$AAR?$AAE?$AAS?$AAE?$AAT?$AA?5?$AAf?$AAa?$AAi?$AAl?$AAe?$AAd?$AA?$AA@FNODOBFM@ 0041cd8c     arcinit.obj
 0001:0001bdae       ??_C@_0DE@GCJLBNBN@?$CK?$CK?5Fail?5to?5iopreset?5the?5adapter?0@FNODOBFM@ 0041cdae     arcinit.obj
 0001:0001bde2       ??_C@_0BI@DKKBLGKC@?$CK?$CK?5IOPReset?5succeeded?4?6?$AA@FNODOBFM@ 0041cde2     arcinit.obj
 0001:0001bdfa       ??_C@_0DB@MLPIECHL@?$CK?5Discard?5HOSTRRQ?5leftover?3?5inde@FNODOBFM@ 0041cdfa     arcinit.obj
 0001:0001be2c       ??_C@_0DG@MCABGJKN@Driver?5should?5not?5work?5under?5MSI@FNODOBFM@ 0041ce2c     arcinit.obj
 0001:0001be62       ??_C@_0DE@DDNIODIO@?$CK?5Set?5pInitStruct?9?$DONoOfMsiVector@FNODOBFM@ 0041ce62     arcinit.obj
 0001:0001be96       ??_C@_0BC@JKJGEENA@leaving?5IOPReset?6?$AA@FNODOBFM@ 0041ce96     arcinit.obj
 0001:0001bea8       ??_C@_0CM@JEPCBIHG@?6entering?5ReinitializeAdapterAft@FNODOBFM@ 0041cea8     arcinit.obj
 0001:0001bed4       ??_C@_0CL@LBAAMMMB@?$CK?$CK?5Adapter?5set?5KERNEL_UP_AND_RUN@FNODOBFM@ 0041ced4     arcinit.obj
 0001:0001bf00       ??_C@_0CH@DPKMOBPP@?$CK?5StorPort?5miniport?5driver?5versi@FNODOBFM@ 0041cf00     arcinit.obj
 0001:0001bf28       ??_C@_0CA@BAOMFHLP@?$CK?5Calling?5InitializeAdapter?4?4?4?6?$AA@FNODOBFM@ 0041cf28     arcinit.obj
 0001:0001bf48       ??_C@_0CE@OJCBEKFM@?$CK?5IopReset?3?5ADAPTER?5NOT?5RUNNING?$CB@FNODOBFM@ 0041cf48     arcinit.obj
 0001:0001bf6c       ??_C@_0CK@PNHBBEHK@leaving?5ReinitializeAdapterAfter@FNODOBFM@ 0041cf6c     arcinit.obj
 0001:0001bf96       ??_C@_0CN@KPEBIFEO@?$CK?5?$DN?$DN?$DN?$DN?$DN?$DN?$DO?5Final?5Vector?5Number?5is@FNODOBFM@ 0041cf96     arcinit.obj
 0001:0001bfc4       ??_C@_0CI@BJJEDHMG@?$CK?5pDeviceExtension?9?$DOVectorCapaci@FNODOBFM@ 0041cfc4     arcinit.obj
 0001:0001bfec       ??_C@_0DE@JJAKLEJD@?$CK?5pDeviceExtension?9?$DOMSIXIoThrott@FNODOBFM@ 0041cfec     arcinit.obj
 0001:0001c020       ??_C@_0DF@LMKAIIEG@?$CK?5pDeviceExtension?9?$DOMSIXIoThrott@FNODOBFM@ 0041d020     arcinit.obj
 0001:0001c056       ??_C@_0BK@OLLEIHIC@?$CK?5Switching?5to?5MSIx?5mode?6?$AA@FNODOBFM@ 0041d056     arcinit.obj
 0001:0001c070       ??_C@_0BA@EAOKKBLN@?$CK?5MSIx?5Enabled?6?$AA@FNODOBFM@ 0041d070     arcinit.obj
 0001:0001c080       ??_C@_0EB@JEEKIEDM@?$CK?5Set?5pInitStruct?9?$DONoOfMsiVector@FNODOBFM@ 0041d080     arcinit.obj
 0001:0001c0c2       ??_C@_0EA@DFHNCIMC@?$CK?5Set?5pInitStruct?9?$DONoOfMsiVector@FNODOBFM@ 0041d0c2     arcinit.obj
 0001:0001c102       ??_C@_0BE@OKKJEBLK@?$CK?5MSIX?5NOT?5Enabled?6?$AA@FNODOBFM@ 0041d102     arcinit.obj
 0001:0001c116       ??_C@_0ED@LLOJEJPI@leaving?5HandleAdapterGetConfig?5a@FNODOBFM@ 0041d116     arcinit.obj
 0001:0001c15a       ??_C@_0EF@MHNEOFPB@?$CK?5leaving?5HandleAdapterGetConfig@FNODOBFM@ 0041d15a     arcinit.obj
 0001:0001c1a0       ??_C@_0DP@PECHNPGJ@leaving?5HandleAdapterGetConfig?5a@FNODOBFM@ 0041d1a0     arcinit.obj
 0001:0001c1e0       ??_C@_0EB@CHAPDLOA@?$CK?5leaving?5HandleAdapterGetConfig@FNODOBFM@ 0041d1e0     arcinit.obj
 0001:0001c222       ??_C@_0EC@JNDOKFCE@leaving?5HandleAdapterCommitConfi@FNODOBFM@ 0041d222     arcinit.obj
 0001:0001c264       ??_C@_0EE@HMHNBLOK@?$CK?5leaving?5HandleAdapterCommitCon@FNODOBFM@ 0041d264     arcinit.obj
 0001:0001c2a8       ??_C@_0CE@FDDAIENL@entering?5HandleAdapterConfigIssu@FNODOBFM@ 0041d2a8     arcinit.obj
 0001:0001c2cc       ??_C@_0EG@EOLGKFDM@leaving?5HandleAdapterConfigIssue@FNODOBFM@ 0041d2cc     arcinit.obj
 0001:0001c312       ??_C@_0EI@BLLNCBDL@?$CK?5leaving?5HandleAdapterConfigIss@FNODOBFM@ 0041d312     arcinit.obj
 0001:0001c35a       ??_C@_0EC@KFDDDOGD@leaving?5HandleAdapterConfigIssue@FNODOBFM@ 0041d35a     arcinit.obj
 0001:0001c39c       ??_C@_0EE@EEHAIAKN@?$CK?5leaving?5HandleAdapterConfigIss@FNODOBFM@ 0041d39c     arcinit.obj
 0001:0001c3e0       ??_C@_0EC@EGKDAAOP@leaving?5HandleAdapterConfigIssue@FNODOBFM@ 0041d3e0     arcinit.obj
 0001:0001c422       ??_C@_0EE@KHOALOCB@?$CK?5leaving?5HandleAdapterConfigIss@FNODOBFM@ 0041d422     arcinit.obj
 0001:0001c466       ??_C@_0CD@FIHDJCJC@leaving?5HandleAdapterConfigIssue@FNODOBFM@ 0041d466     arcinit.obj
 0001:0001c48a       ??_C@_0BM@OLPDNDAC@entering?5InitializeAdapter?6?$AA@FNODOBFM@ 0041d48a     arcinit.obj
 0001:0001c4a6       ??_C@_1DA@HBPONGDO@?$AAF?$AAa?$AAi?$AAl?$AAe?$AAd?$AA?5?$AAt?$AAo?$AA?5?$AAs?$AAt?$AAa?$AAr?$AAt?$AA?5?$AAA?$AAd?$AAa?$AAp?$AAt?$AAe?$AAr?$AA?$AA@FNODOBFM@ 0041d4a6     arcinit.obj
 0001:0001c4d6       ??_C@_0CP@OADFCMNE@leaving?5InitializeAdapter?3?5fail?5@FNODOBFM@ 0041d4d6     arcinit.obj
 0001:0001c506       ??_C@_0DB@CKIIOBC@?$CK?5leaving?5InitializeAdapter?3?5fai@FNODOBFM@ 0041d506     arcinit.obj
 0001:0001c538       ??_C@_0BL@CPLHAEBI@leaving?5InitializeAdapter?6?$AA@FNODOBFM@ 0041d538     arcinit.obj
 0001:0001c554       ??_C@_0BK@LNIBADPE@?$CK?5Setting?5StatusBatching?6?$AA@FNODOBFM@ 0041d554     arcinit.obj
 0001:0001c56e       ??_C@_0EF@JDALIICL@?$CK?5Firmware?5should?5support?5ACI2?5i@FNODOBFM@ 0041d56e     arcinit.obj
 0001:0001c5b4       ??_C@_0CB@DDHFLEBF@?$CK?5FW?5sets?5KERNEL_UP_AND_RUNNING?6@FNODOBFM@ 0041d5b4     arcinit.obj
 0001:0001c5d6       ??_C@_0CC@HECBNNJJ@?$CK?5FW?5is?5ready?5for?5config?5command@FNODOBFM@ 0041d5d6     arcinit.obj
 0001:0001c5f8       ??_C@_0BJ@GODFBPEB@?$CK?5Get?5config?5from?5FW?5ok?6?$AA@FNODOBFM@ 0041d5f8     arcinit.obj
 0001:0001c612       ??_C@_0BK@PANMBLHC@?$CK?5Commit?5config?5to?5FW?5ok?6?$AA@FNODOBFM@ 0041d612     arcinit.obj
 0001:0001c62c       ??_C@_0CA@BDIKNGAL@?$CK?5INIT?5Structure?5sent?5to?5FW?5ok?6?$AA@FNODOBFM@ 0041d62c     arcinit.obj
 0001:0001c64c       ??_C@_0BK@HCHBCLAI@?$CK?5Get?5FW?5debug?5buffer?5ok?6?$AA@FNODOBFM@ 0041d64c     arcinit.obj
 0001:0001c666       ??_C@_0BO@IEENCLHE@entering?5HwInitializeAdapter?6?$AA@FNODOBFM@ 0041d666     arcinit.obj
 0001:0001c684       ??_C@_1CA@OFEHMOBK@?$AAB?$AAa?$AAd?$AA?5?$AAP?$AAo?$AAr?$AAt?$AA?5?$AAD?$AAr?$AAi?$AAv?$AAe?$AAr?$AA?$AA@FNODOBFM@ 0041d684     arcinit.obj
 0001:0001c6a4       ??_C@_0BO@FHHBMMGN@?$CK?5PerfConfigData?4Flags?3?50x?$CFx?6?$AA@FNODOBFM@ 0041d6a4     arcinit.obj
 0001:0001c6c2       ??_C@_0CF@FDBIIPFF@?$CK?5This?5Tupelo?5driver?5is?5MSI?5enab@FNODOBFM@ 0041d6c2     arcinit.obj
 0001:0001c6e8       ??_C@_0EH@ONHPKJKD@?$CK?5StorPortGetMSIInfo?5returned?5Fa@FNODOBFM@ 0041d6e8     arcinit.obj
 0001:0001c730       ??_C@_0EC@KLPNNIKH@?$CK?5StorPortGetMSIInfo?5returned?5st@FNODOBFM@ 0041d730     arcinit.obj
 0001:0001c772       ??_C@_0EE@OLLCNNAO@?$CK?5StorPortGetMSIInfo?5returned?5st@FNODOBFM@ 0041d772     arcinit.obj
 0001:0001c7b6       ??_C@_0EJ@OBPFJGIJ@?$CK?5StorPortGetMSIInfo?5returned?5st@FNODOBFM@ 0041d7b6     arcinit.obj
 0001:0001c800       ??_C@_0FE@LBLIGLIO@GetDoorbellMaskForIOPReset?5retur@FNODOBFM@ 0041d800     arcinit.obj
 0001:0001c854       ??_C@_0DN@IMFNPMPP@?$CK?5Failed?5to?5Initialize?5Adapter?5i@FNODOBFM@ 0041d854     arcinit.obj
 0001:0001c892       ??_C@_0DE@CMNGFMDL@?$CK?5Succeed?5to?5Initialize?5Adapter?5@FNODOBFM@ 0041d892     arcinit.obj
 0001:0001c8c6       ??_C@_0EG@KGJBNOFG@?$CK?5Failed?5to?5Initialize?5Adapter?5i@FNODOBFM@ 0041d8c6     arcinit.obj
 0001:0001c90c       ??_C@_0DA@GDJCAINB@?$CK?5Succeed?5to?5Initialize?5Adapter?5@FNODOBFM@ 0041d90c     arcinit.obj
 0001:0001c93c       ??_C@_0BI@BOGNCAIA@entering?5InitializeDPC?6?$AA@FNODOBFM@ 0041d93c     arcinit.obj
 0001:0001c954       ??_C@_0DJ@MGMHFMAN@?$CK?5Failed?5to?5Initialize?5Adapter?5i@FNODOBFM@ 0041d954     arcinit.obj
 0001:0001c98e       ??_C@_0BJ@CFFELFMJ@?$CK?5MSIx?5DPCs?5initialized?6?$AA@FNODOBFM@ 0041d98e     arcinit.obj
 0001:0001c9a8       ??_C@_0BJ@IKFKIDCM@?$CK?5?9?5Done?5InitializeDPC?5?6?$AA@FNODOBFM@ 0041d9a8     arcinit.obj
 0001:0001c9c2       ??_C@_0BH@PAHICDNJ@leaving?5InitializeDPC?6?$AA@FNODOBFM@ 0041d9c2     arcinit.obj
 0001:0001c9da       ??_C@_0CP@OJKLKHLO@entering?5InitializeConsumerProdu@FNODOBFM@ 0041d9da     arcinit.obj
 0001:0001ca0a       ??_C@_0DE@MJJEGAKI@leaving?5InitializeConsumerProduc@FNODOBFM@ 0041da0a     arcinit.obj
 0001:0001ca3e       ??_C@_0CO@NEGLFCOP@leaving?5InitializeConsumerProduc@FNODOBFM@ 0041da3e     arcinit.obj
 0001:0001ca6c       ??_C@_0CP@IKCNDLML@entering?5InitializeConsumerProdu@FNODOBFM@ 0041da6c     arcinit.obj
 0001:0001ca9c       ??_C@_0DF@IICIHNDP@leaving?5InitializeConsumerProduc@FNODOBFM@ 0041da9c     arcinit.obj
 0001:0001cad2       ??_C@_0DE@OBANPGHF@leaving?5InitializeConsumerProduc@FNODOBFM@ 0041dad2     arcinit.obj
 0001:0001cb06       ??_C@_0CP@GDFIJJML@entering?5InitializeMessageUnitQu@FNODOBFM@ 0041db06     arcinit.obj
 0001:0001cb36       ??_C@_0DF@CLHHLLI@leaving?5InitializeMessageUnitQue@FNODOBFM@ 0041db36     arcinit.obj
 0001:0001cb6c       ??_C@_0DE@BBDIIBAC@leaving?5InitializeMessageUnitQue@FNODOBFM@ 0041db6c     arcinit.obj
 0001:0001cba0       ??_C@_0BI@PNFIHJKN@entering?5MapDeviceBase?6?$AA@FNODOBFM@ 0041dba0     arcinit.obj
 0001:0001cbb8       ??_C@_1CM@FGGDGCGC@?$AAA?$AAd?$AAa?$AAp?$AAt?$AAe?$AAr?$AA?5?$AAb?$AAo?$AAo?$AAt?$AA?5?$AAt?$AAi?$AAm?$AAe?$AA?5?$AAo?$AAu?$AAt?$AA?$AA@FNODOBFM@ 0041dbb8     arcinit.obj
 0001:0001cbe4       ??_C@_0DG@EECBHNEJ@?$CK?5Driver?5did?5not?5get?564?5bit?5FIB?5@FNODOBFM@ 0041dbe4     arcinit.obj
 0001:0001cc1a       ??_C@_0DL@HHJHAPNC@?$CK?5StorPortGetDeviceBase?5failed?0?5@FNODOBFM@ 0041dc1a     arcinit.obj
 0001:0001cc56       ??_C@_0FM@FAGAFMJI@?$CK?5StorPortGetDeviceBaseB1?5failed@FNODOBFM@ 0041dc56     arcinit.obj
 0001:0001ccb2       ??_C@_0FM@DFFNMELK@?$CK?5StorPortGetDeviceBaseB0?5failed@FNODOBFM@ 0041dcb2     arcinit.obj
 0001:0001cd0e       ??_C@_0DH@GMHBCEJM@?$CK?5GET_MINIARC_PROPERTIES?5fails?0?5@FNODOBFM@ 0041dd0e     arcinit.obj
 0001:0001cd46       ??_C@_0CE@JIIGOPEA@?$CK?5This?5is?5a?5BEDROC?5inplementatio@FNODOBFM@ 0041dd46     arcinit.obj
 0001:0001cd6a       ??_C@_0CF@HKNELPOC@leaving?5MapDeviceBase?5?9?5rtnval?5?$DN@FNODOBFM@ 0041dd6a     arcinit.obj
 0001:0001cd90       ??_C@_0BG@LOIMFNHP@entering?5MatchPciIds?6?$AA@FNODOBFM@ 0041dd90     arcinit.obj
 0001:0001cda6       ??_C@_08HNOCAICB@Adaptec?5?$AA@FNODOBFM@ 0041dda6     arcinit.obj
 0001:0001cdb0       ??_C@_0CC@GEDCIDMJ@leaving?5MatchPciIds?0?5rtnval?5?$DN?5?$CFx@FNODOBFM@ 0041ddb0     arcinit.obj
 0001:0001cdd2       ??_C@_0DG@MJCHKBMN@?$CK?5Calling?5CompleteBufferedReques@FNODOBFM@ 0041ddd2     arcinit.obj
 0001:0001ce08       ??_C@_0HF@LDMKNKBL@?$CK?5Calling?5DequeueRawIoReadWriteR@FNODOBFM@ 0041de08     arcinit.obj
 0001:0001ce7e       ??_C@_0DO@HDLNLCMA@?$CK?5Calling?5CompleteAllSortingQueu@FNODOBFM@ 0041de7e     arcinit.obj
 0001:0001cebc       ??_C@_0CG@EHFONFB@ReturningLocalOutstandingRequest@FNODOBFM@ 0041debc     arcinit.obj
 0001:0001cee2       ??_C@_0CL@CGNJGHDF@?$CK?5?$CFd?5outstanding?5IO?5left?5after?5c@FNODOBFM@ 0041dee2     arcinit.obj
 0001:0001cf0e       ??_C@_0CF@IKJOOFLA@?$CK?5ResetAdapter?3?5Entering?5Routine@FNODOBFM@ 0041df0e     arcinit.obj
 0001:0001cf34       ??_C@_0FI@OABPGHMC@?$CK?5ResetAdapter?3?5FW?5is?5processing@FNODOBFM@ 0041df34     arcinit.obj
 0001:0001cf8c       ??_C@_0DK@DMNFFNOF@?$CK?5ResetAdapter?3?5OS?5calls?5ResetAd@FNODOBFM@ 0041df8c     arcinit.obj
 0001:0001cfc6       ??_C@_0CE@IFPMEIEL@?$CK?5ResetAdapter?3?5BlinLed?5Code?3?50x@FNODOBFM@ 0041dfc6     arcinit.obj
 0001:0001cfea       ??_C@_1CE@ENBAPEOO@?$AAB?$AAl?$AAi?$AAn?$AAk?$AAL?$AAE?$AAD?$AA?5?$AAd?$AAe?$AAt?$AAe?$AAc?$AAt?$AAe?$AAd?$AA?$AA@FNODOBFM@ 0041dfea     arcinit.obj
 0001:0001d00e       ??_C@_0CL@MJAGNJPB@?$CK?5ResetAdapter?3?5IOP?5RESET?5due?5to@FNODOBFM@ 0041e00e     arcinit.obj
 0001:0001d03a       ??_C@_0DG@CLNGJPOA@?$CK?5ResetAdapter?3?5SendSynchFib?5fai@FNODOBFM@ 0041e03a     arcinit.obj
 0001:0001d070       ??_C@_0FF@JLPFKNGK@?$CK?5ResetAdapter?3?5There?5is?5a?5pendi@FNODOBFM@ 0041e070     arcinit.obj
 0001:0001d0c6       ??_C@_0EC@MMLNJELN@?$CK?5ResetAdapter?3?5set?5TriggerIOPRe@FNODOBFM@ 0041e0c6     arcinit.obj
 0001:0001d108       ??_C@_0EH@BGKKNIMJ@?$CK?5ResetAdapter?3?5synch?5command?5Re@FNODOBFM@ 0041e108     arcinit.obj
 0001:0001d150       ??_C@_0EE@KPCKIKGP@?$CK?5ResetAdapter?3?5AdapterIsAlive?5r@FNODOBFM@ 0041e150     arcinit.obj
 0001:0001d194       ??_C@_0DN@OJOIDCGM@?$CK?5ResetAdapter?3?5leaving?5Routine?5@FNODOBFM@ 0041e194     arcinit.obj
 0001:0001d1d2       ??_C@_0DN@MKLLHNDH@?$CK?5ResetAdapter?3?5IOP?5RESET?5due?5to@FNODOBFM@ 0041e1d2     arcinit.obj
 0001:0001d210       ??_C@_0DA@IHJFMKGH@?$CK?5ResetAdapter?3?5IOP?5RESET?5due?5to@FNODOBFM@ 0041e210     arcinit.obj
 0001:0001d240       ??_C@_0FK@LPHHHNGK@?$CK?5ResetAdapter?3?5device?5on?5path?54@FNODOBFM@ 0041e240     arcinit.obj
 0001:0001d29a       ??_C@_0EG@FKMCGCCN@?$CK?5ResetAdapter?3?5IOP?5RESET?5due?5to@FNODOBFM@ 0041e29a     arcinit.obj
 0001:0001d2e0       ??_C@_0DE@IDNFNJBF@?$CK?5ResetAdapter?3?5NO?5lun?5reset?5cou@FNODOBFM@ 0041e2e0     arcinit.obj
 0001:0001d314       ??_C@_0DM@KJNOMFJC@?$CK?5ResetAdapter?3?5leaving?5Routine?0@FNODOBFM@ 0041e314     arcinit.obj
 0001:0001d350       ??_C@_0EK@OOPLAGOO@?$CK?5ResetAdapter?3?5set?5timer?5to?5che@FNODOBFM@ 0041e350     arcinit.obj
 0001:0001d39a       ??_C@_0DM@LMPLKKMJ@?$CK?5ResetAdapter?3?5leaving?5Routine?5@FNODOBFM@ 0041e39a     arcinit.obj
 0001:0001d3d6       ??_C@_0DB@KLKDBGPC@?$CK?5current?5ElapsedTime?5is?5?$CFx?4?5Dri@FNODOBFM@ 0041e3d6     arcinit.obj
 0001:0001d408       ??_C@_0DB@LKKOAGAA@?$CK?$CK?5Send?5Synch?5Command?5VM_SetDynA@FNODOBFM@ 0041e408     arcinit.obj
 0001:0001d43a       ??_C@_0CP@HANMIEGD@?$CK?5Set?5Dynamic?5Adapter?5Properties@FNODOBFM@ 0041e43a     arcinit.obj
 0001:0001d46a       ??_C@_0BP@IBJHMEIL@?$CK?5?5HBA?5Cntrl?5Function?5Mode?5?$CFx?6?$AA@FNODOBFM@ 0041e46a     arcinit.obj
 0001:0001d48a       ??_C@_0ED@KLKEOEFE@?$CK?5GetHbaPhyDevInfo?3?5Send?5Synch?5C@FNODOBFM@ 0041e48a     arcinit.obj
 0001:0001d4ce       ??_C@_0EJ@GAJDFDIF@?$CK?5GetHbaPhyDevInfo?3?5CT_GET_PHYDE@FNODOBFM@ 0041e4ce     arcinit.obj
 0001:0001d518       ??_C@_0DK@BCAHFDGL@?$CK?5GetHbaPhyDevInfo?3?5Send?5Synch?5C@FNODOBFM@ 0041e518     arcinit.obj
 0001:0001d552       ??_C@_0EF@NNHICAHG@?$CK?5GetHbaPhyDevInfo?3?5Sync?5Command@FNODOBFM@ 0041e552     arcinit.obj
 0001:0001d598       ??_C@_0DM@IJMGIHKF@?$CK?5GetHbaPhyDevInfo?3?5Send?5Synch?5C@FNODOBFM@ 0041e598     arcinit.obj
 0001:0001d5d4       ??_C@_0DP@EPCIGAGM@?$CK?5GetHbaPhyDevInfo?3?5Received?5Wro@FNODOBFM@ 0041e5d4     arcinit.obj
 0001:0001d614       ??_C@_0FE@NKLEACGL@?$CK?5ConfigHBADeviceInit?3?5PHY_DEV_I@FNODOBFM@ 0041e614     arcinit.obj
 0001:0001d668       ??_C@_0FC@CEEDMHOD@?$CK?5ConfigHBADeviceInit?3?5PHY_DEV_I@FNODOBFM@ 0041e668     arcinit.obj
 0001:0001d6ba       ??_C@_0DJ@IHGLCMIF@?$CK?5ConfigHBADeviceInit?3?5not?5a?5HBA@FNODOBFM@ 0041e6ba     arcinit.obj
 0001:0001d6f4       ??_C@_0EH@EBMPFNCB@?$CK?5GetHbaPhyDevList?3?5Send?5Synch?5C@FNODOBFM@ 0041e6f4     arcinit.obj
 0001:0001d73c       ??_C@_0DG@BDNFILEO@?$CK?5GetHbaPhyDevList?3?5CT_GET_PHYDE@FNODOBFM@ 0041e73c     arcinit.obj
 0001:0001d772       ??_C@_0DM@GKMMKGOD@?$CK?5GetHbaPhyDevList?3?5CT_GET_PHYDE@FNODOBFM@ 0041e772     arcinit.obj
 0001:0001d7ae       ??_C@_0EO@PACGLEM@?$CK?5GetHbaPhyDevList?3?5Synch?5Comman@FNODOBFM@ 0041e7ae     arcinit.obj
 0001:0001d7fc       ??_C@_0EF@LCIPIHKL@?$CK?5GetHbaPhyDevList?3?5Send?5Synch?5C@FNODOBFM@ 0041e7fc     arcinit.obj
 0001:0001d842       ??_C@_0EF@BPBMMFO@?$CK?5GetHbaPhyDevList?3?5Send?5Synch?5C@FNODOBFM@ 0041e842     arcinit.obj
 0001:0001d888       ??_C@_0EB@GDJIECLG@?$CK?5GetHbaPhyDevList?3?5Send?5Synch?5C@FNODOBFM@ 0041e888     arcinit.obj
 0001:0001d8ca       ??_C@_0DP@EPPGCKNK@?$CK?5GetHbaPhyDevList?3?5Received?5Wro@FNODOBFM@ 0041e8ca     arcinit.obj
 0001:0001d90a       ??_C@_0FM@KMPOIDHC@?$CK?5ScanMapTblForCheck?3?5found?5Devi@FNODOBFM@ 0041e90a     arcinit.obj
 0001:0001d966       ??_C@_0CN@HJFDOJDA@?$CK?5ScanMapTblForCheck?3?5not?5a?5HBA?5@FNODOBFM@ 0041e966     arcinit.obj
 0001:0001d994       ??_C@_0DN@KPJLDPIL@?$CK?5ScanMapTblForCheck?3?5not?5a?5HBA?5@FNODOBFM@ 0041e994     arcinit.obj
 0001:0001d9d2       ??_C@_0DJ@MNJIDJF@?$CK?5ScanMapTblForCheck?3?5found?5new?5@FNODOBFM@ 0041e9d2     arcinit.obj
 0001:0001da0c       ??_C@_0DH@DENBGCND@?$CK?5ScanMapTblForCheck?3?5found?5new?5@FNODOBFM@ 0041ea0c     arcinit.obj
 0001:0001da44       ??_C@_0EM@OADFOJJH@?$CK?5ScanMapTblForDeviceAdd?3?5add?5ne@FNODOBFM@ 0041ea44     arcinit.obj
 0001:0001da90       ??_C@_0DM@IBDHLPON@?$CK?5ScanMapTblForDeviceAdd?3?5not?5a?5@FNODOBFM@ 0041ea90     arcinit.obj
 0001:0001dacc       ??_C@_0EK@NGDDIFNC@?$CK?5ScanMapTblForDeviceAdd?3?5add?5ne@FNODOBFM@ 0041eacc     arcinit.obj
 0001:0001db16       ??_C@_0EN@LKFFLIBM@?$CK?5ScanMapTblForDeviceAdd?3?5not?5a?5@FNODOBFM@ 0041eb16     arcinit.obj
 0001:0001db64       ??_C@_1EK@IBCIJFDK@?$AAR?$AAe?$AAs?$AAe?$AAt?$AA?5?$AAf?$AAr?$AAo?$AAm?$AA?5?$AAO?$AAS?$AA?3?$AAp?$AAa?$AAt?$AAh?$AA?5?$AA?$CD?$AA?5?$AA?5?$AA?0?$AAo?$AAu?$AAt?$AAs?$AAt?$AAa?$AAn?$AAd?$AAi@FNODOBFM@ 0041eb64     arcinit.obj
 0001:0001dbae       ??_C@_1EK@PDIMAHFB@?$AAG?$AAo?$AAt?$AA?5?$AAL?$AAU?$AAN?$AA?5?$AAR?$AAE?$AAS?$AAE?$AAT?$AA?5?$AAf?$AAo?$AAr?$AA?5?$AAp?$AAa?$AAt?$AAh?$AA?5?$AA?$CD?$AA?5?$AA?5?$AA?0?$AA?5?$AAt?$AAa?$AAr?$AAg@FNODOBFM@ 0041ebae     arcinit.obj
 0001:0001dbf8       ??_C@_1FA@GAKKMNHF@?$AAG?$AAo?$AAt?$AA?5?$AAT?$AAa?$AAr?$AAg?$AAe?$AAt?$AA?5?$AAR?$AAE?$AAS?$AAE?$AAT?$AA?5?$AAf?$AAo?$AAr?$AA?5?$AAp?$AAa?$AAt?$AAh?$AA?5?$AA?$CD?$AA?5?$AA?5?$AA?0?$AA?5?$AAt@FNODOBFM@ 0041ebf8     arcinit.obj
 0001:0001dc48       ??_C@_1EC@DEFLMBHE@?$AAI?$AAO?$AAP?$AA?5?$AAR?$AAE?$AAS?$AAE?$AAT?$AA?5?$AAb?$AAe?$AAc?$AAa?$AAu?$AAs?$AAe?$AA?5?$AAo?$AAf?$AA?5?$AAF?$AAW?$AA?5?$AAB?$AAl?$AAi?$AAn?$AAk?$AAL?$AAE?$AAD@FNODOBFM@ 0041ec48     arcinit.obj
 0001:0001dc8a       ??_C@_1FA@GLBMBCFD@?$AAR?$AAe?$AAq?$AAu?$AAe?$AAs?$AAt?$AAA?$AAd?$AAa?$AAp?$AAt?$AAe?$AAr?$AAI?$AAn?$AAf?$AAo?$AA?5?$AAp?$AAe?$AAn?$AAd?$AAi?$AAn?$AAg?$AA?5?$AA?5?$AA?5?$AA?5?$AA?5?$AA?5@FNODOBFM@ 0041ec8a     arcinit.obj
 0001:0001dcda       ??_C@_1EK@DPFNMDNI@?$AAI?$AAO?$AAP?$AAR?$AAE?$AAS?$AAE?$AAT?$AA?3?$AA?5?$AAR?$AAe?$AAq?$AAu?$AAe?$AAs?$AAt?$AAA?$AAd?$AAa?$AAp?$AAt?$AAe?$AAr?$AAI?$AAn?$AAf?$AAo?$AA?5?$AAt?$AAi?$AAm@FNODOBFM@ 0041ecda     arcinit.obj
 0001:0001dd24       ??_C@_1EC@JONMGECF@?$AAR?$AAA?$AA?3?$AA?5?$AAA?$AAd?$AAa?$AAp?$AAt?$AAe?$AAr?$AAI?$AAs?$AAA?$AAl?$AAi?$AAv?$AAe?$AA?5?$AAr?$AAe?$AAt?$AAu?$AAr?$AAn?$AAs?$AA?5?$AAf?$AAa?$AAl?$AAs?$AAe@FNODOBFM@ 0041ed24     arcinit.obj
 0001:0001dd66       ??_C@_1DM@LFFFLHNF@?$AAI?$AAO?$AAP?$AA?5?$AAR?$AAE?$AAS?$AAE?$AAT?$AA?5?$AAf?$AAo?$AAr?$AA?5?$AAS?$AAm?$AAa?$AAr?$AAt?$AAH?$AAB?$AAA?$AA?5?$AAp?$AAa?$AAt?$AAh?$AA?5?$AA?$CD?$AA?$AA@FNODOBFM@ 0041ed66     arcinit.obj
 0001:0001dda2       ??_C@_1EK@EBJJOFBF@?$AAR?$AAE?$AAS?$AAE?$AAT?$AA?$CI?$AAc?$AAn?$AAt?$AA?$DO?$AA?$DN?$AA5?$AA?$CJ?$AA?3?$AA?5?$AAp?$AAa?$AAt?$AAh?$AA?5?$AA?$CD?$AA?5?$AA?5?$AA?0?$AA?5?$AAt?$AAa?$AAr?$AAg?$AAe?$AAt?$AA?5@FNODOBFM@ 0041eda2     arcinit.obj
 0001:0001ddec       ??_C@_0BG@FGBHCKJG@CompleteQueuedRequest?$AA@FNODOBFM@ 0041edec     cmddelivery.obj
 0001:0001de02       ??_C@_0DM@OFFCECMD@IN?5?$CFs?0?5WE?5ARE?5SEEING?5AIF?5FIB?4?5DO@FNODOBFM@ 0041ee02     cmddelivery.obj
 0001:0001de3e       ??_C@_0L@ENAJINDB@Management?$AA@FNODOBFM@ 0041ee3e     cmddelivery.obj
 0001:0001de4a       ??_C@_0BB@JIADCMFJ@Array?5?5?5?5?5?5?5?5?5?5?5?$AA@FNODOBFM@ 0041ee4a     cmddelivery.obj
 0001:0001de5c       ??_C@_08BFDLJAAH@ADAPTEC?5?$AA@FNODOBFM@ 0041ee5c     cmddelivery.obj
 0001:0001de66       ??_C@_0BB@HJODFKJH@ARRAY?5?5?5?5?5?5?5?5?5?5?5?$AA@FNODOBFM@ 0041ee66     cmddelivery.obj
 0001:0001de78       ??_C@_0FM@ENJACBOF@?$CK?5SCSIOP_SYNCHRONIZE_CACHE?$CICDM?$CJ?3@FNODOBFM@ 0041ee78     cmddelivery.obj
 0001:0001ded4       ??_C@_0GA@MEOEEOJH@?$CK?5SCSIOP_SYNCHRONIZE_CACHE?$CICDM?$CJ?3@FNODOBFM@ 0041eed4     cmddelivery.obj
 0001:0001df34       ??_C@_0HI@CALKOMHC@?$CK?5SendSynchFib?3?5There?5is?5a?5pendi@FNODOBFM@ 0041ef34     cmddelivery.obj
 0001:0001dfac       ??_C@_0CB@IIENMBOI@?$CK?5Got?5an?5AIF?5in?5crash?5dump?5mode?6@FNODOBFM@ 0041efac     cmddelivery.obj
 0001:0001dfce       ??_C@_0DO@NPBDNHBG@?$CK?5Should?5not?5be?5here?0?5we?5should?5@FNODOBFM@ 0041efce     cmddelivery.obj
 0001:0001e00c       ??_C@_0CO@PDPAIINM@?$CK?5PollSmartHBAFIBCompletion?3?5wai@FNODOBFM@ 0041f00c     cmddelivery.obj
 0001:0001e03a       ??_C@_0FM@IHOMFPBM@?$CK?5In?5StartIo?0?5FW?5is?5still?5NOT?5ba@FNODOBFM@ 0041f03a     cmddelivery.obj
 0001:0001e096       ??_C@_0CN@EPOHBMBH@?$CK?5path?5?$CFd?5target?5?$CFd?5reset?5counte@FNODOBFM@ 0041f096     cmddelivery.obj
 0001:0001e0c4       ??_C@_0CB@KIAHGGON@?5RESET?5is?5for?5Smart?5HBA?5device?5?6@FNODOBFM@ 0041f0c4     cmddelivery.obj
 0001:0001e0e6       ??_C@_0BP@PAHACOBL@?$CK?5Got?5path?5?$CFd?5target?5?$CFd?5reset?6?$AA@FNODOBFM@ 0041f0e6     cmddelivery.obj
 0001:0001e106       ??_C@_0CC@BGHDODBG@?$CK?5SRB_FUNCTION_POWER?3?5action?3?5?$CFd@FNODOBFM@ 0041f106     cmddelivery.obj
 0001:0001e128       ??_C@_0BP@DFKLHFDI@?$CK?5SRB_FUNCTION_POWER?3?5sleep?51?6?$AA@FNODOBFM@ 0041f128     cmddelivery.obj
 0001:0001e148       ??_C@_0DL@PCKMOFFE@?$CK?5SRB_FUNCTION_POWER?3?5coming?5bac@FNODOBFM@ 0041f148     cmddelivery.obj
 0001:0001e184       ??_C@_0CG@NCNALCOB@?$CK?5SRB_FUNCTION_POWER?3?5going?5to?5S@FNODOBFM@ 0041f184     cmddelivery.obj
 0001:0001e1aa       ??_C@_0CA@IBGDOHDE@?$CK?5SRB_FUNCTION_POWER?3?5shutdown?6?$AA@FNODOBFM@ 0041f1aa     cmddelivery.obj
 0001:0001e1ca       ??_C@_0CD@NOANDIPK@?$CK?5SRB_FUNCTION_POWER?3?5shutdownOf@FNODOBFM@ 0041f1ca     cmddelivery.obj
 0001:0001e1ee       ??_C@_0BO@KPPCGIPP@?$CK?5SRB_FUNCTION_POWER?3?5reboot?6?$AA@FNODOBFM@ 0041f1ee     cmddelivery.obj
 0001:0001e20c       ??_C@_0BJ@NDPKABON@entering?5AdapterControl?6?$AA@FNODOBFM@ 0041f20c     cmdproc.obj
 0001:0001e226       ??_C@_0CF@FDIANAIH@?$CK?5?9?5AdapterControl?3?5ScsiStopAdap@FNODOBFM@ 0041f226     cmdproc.obj
 0001:0001e24c       ??_C@_0FJ@DLLPOCIO@?$CK?5?9?5AdapterControl?3?5ScsiStopAdap@FNODOBFM@ 0041f24c     cmdproc.obj
 0001:0001e2a6       ??_C@_0DK@JIECJOFO@?$CK?5Set?5pInitStruct?9?$DONoOfMsiVector@FNODOBFM@ 0041f2a6     cmdproc.obj
 0001:0001e2e0       ??_C@_0HA@BIJAMPMG@?$CK?5?9?5AdapterControl?3?5ScsiSetBootC@FNODOBFM@ 0041f2e0     cmdproc.obj
 0001:0001e350       ??_C@_0DL@CMAPNHGC@?$CK?5?9?5AdapterControl?3?5ScsiSetBootC@FNODOBFM@ 0041f350     cmdproc.obj
 0001:0001e38c       ??_C@_0DI@IPKKLNPP@?$CK?5?9?5AdapterControl?3?5ScsiSetBootC@FNODOBFM@ 0041f38c     cmdproc.obj
 0001:0001e3c4       ??_C@_0HE@CIFLMEO@?$CK?5?9?5AdapterControl?3?5ScsiSetRunni@FNODOBFM@ 0041f3c4     cmdproc.obj
 0001:0001e438       ??_C@_0CI@NDPGKLNN@?$CK?5?9?5AdapterControl?3?5ScsiRestartA@FNODOBFM@ 0041f438     cmdproc.obj
 0001:0001e460       ??_C@_0CM@CNGCOMHH@?$CK?5Before?5checking?5Adapter?5Health@FNODOBFM@ 0041f460     cmdproc.obj
 0001:0001e48c       ??_C@_0BF@GMFKAGLA@?$CK?$CK?5BlinLed?5Code?3?5?$CFx?6?$AA@FNODOBFM@ 0041f48c     cmdproc.obj
 0001:0001e4a2       ??_C@_0DM@EBNPFHJD@?$CK?5set?5timer?5to?5check?5the?5FW?5stat@FNODOBFM@ 0041f4a2     cmdproc.obj
 0001:0001e4de       ??_C@_0CM@LGOLDMAP@?$CK?5leaving?5AdapterControl?5Routine@FNODOBFM@ 0041f4de     cmdproc.obj
 0001:0001e50a       ??_C@_0GP@BJCLBBHJ@?$CK?5CHECK_ADAPTER_HEALTH?5failed?0?5s@FNODOBFM@ 0041f50a     cmdproc.obj
 0001:0001e57a       ??_C@_0GI@HKBIHHID@?$CK?5START_ADAPTER?5failed?0?5start?5a?5@FNODOBFM@ 0041f57a     cmdproc.obj
 0001:0001e5e2       ??_C@_0CO@CEANCDOF@?$CK?5?9?5AdapterControl?3?5Reset?5HostRR@FNODOBFM@ 0041f5e2     cmdproc.obj
 0001:0001e610       ??_C@_0EF@CJJLGBJF@?$CK?5Start?5a?5timer?5to?5update?5Contai@FNODOBFM@ 0041f610     cmdproc.obj
 0001:0001e656       ??_C@_0EG@HNFCBHB@?$CK?5Start?5a?5timer?5to?5update?5Contai@FNODOBFM@ 0041f656     cmdproc.obj
 0001:0001e69c       ??_C@_0CN@OHJICFOG@?$CK?5?9?5AdapterControl?3?5ScsiQuery?5wi@FNODOBFM@ 0041f69c     cmdproc.obj
 0001:0001e6ca       ??_C@_0DA@CMHNEFAA@?$CK?5?9?5AdapterControl?3?5ScsiQuery?5WI@FNODOBFM@ 0041f6ca     cmdproc.obj
 0001:0001e6fa       ??_C@_0DB@DKFDCCOB@?$CK?5Unsupported?5AdapterControl?5cod@FNODOBFM@ 0041f6fa     cmdproc.obj
 0001:0001e72c       ??_C@_0BI@MBKDPNLO@leaving?5AdapterControl?6?$AA@FNODOBFM@ 0041f72c     cmdproc.obj
 0001:0001e744       ??_C@_0CO@NKBJPPMA@?$CK?5buildio?3?5LBA?5OUT?5OF?5RANGE?0?5sen@FNODOBFM@ 0041f744     cmdproc.obj
 0001:0001e772       ??_C@_0FN@LKLFGDKL@?$CK?5buildio?3?5LBA?5OUT?5OF?5RANGE?0?5sen@FNODOBFM@ 0041f772     cmdproc.obj
 0001:0001e7d0       ??_C@_0FA@MOKLGDID@?$CK?5buildio?3?5LBA?5OUT?5OF?5RANGE?0?5sen@FNODOBFM@ 0041f7d0     cmdproc.obj
 0001:0001e820       ??_C@_0GA@IGOANHED@?$CK?5buildio?3?5LBA?5OUT?5OF?5RANGE?0?5sen@FNODOBFM@ 0041f820     cmdproc.obj
 0001:0001e880       ??_C@_0DM@NPKIKBA@?$CK?5IOP?5RESET?5is?5done?5in?5ProcessIo@FNODOBFM@ 0041f880     ioctl.obj
 0001:0001e8bc       ??_C@_0DL@IOLCNFHG@?$CK?5IOP?5RESET?5failed?5in?5ProcessIoc@FNODOBFM@ 0041f8bc     ioctl.obj
 0001:0001e8f8       ??_C@_07MPDDHOMN@CSMIALL?$AA@FNODOBFM@ 0041f8f8     ioctl.obj
 0001:0001e900       ??_C@_07OODOBGKD@CSMIARY?$AA@FNODOBFM@ 0041f900     ioctl.obj
 0001:0001e908       ??_C@_07PAKBHMBE@CSMISAS?$AA@FNODOBFM@ 0041f908     ioctl.obj
 0001:0001e910       ??_C@_07BHCKAAPP@CSMIPHY?$AA@FNODOBFM@ 0041f910     ioctl.obj
 0001:0001e918       ??_C@_0DF@CHPLNPBM@?$CK?5ProcessIoctl?3?5Internal?5Print?5B@FNODOBFM@ 0041f918     ioctl.obj
 0001:0001e94e       ??_C@_0CE@NGAHOGLJ@?$CK?5ProcessIoctl?3?5private?5cdb?8s?5he@FNODOBFM@ 0041f94e     ioctl.obj
 0001:0001e972       ??_C@_0CH@HPKPAOCF@?$CK?5ProcessIoctl?3?5DBG_IO_TRACE?5fla@FNODOBFM@ 0041f972     ioctl.obj
 0001:0001e99a       ??_C@_0CK@OFFABCEM@?$CK?5ProcessIoctl?3?5DBG_IOCTL_TRACE?5@FNODOBFM@ 0041f99a     ioctl.obj
 0001:0001e9c4       ??_C@_0CM@CGIIOCGI@?$CK?5ProcessIoctl?3?5DBG_CLUSTER_TRAC@FNODOBFM@ 0041f9c4     ioctl.obj
 0001:0001e9f0       ??_C@_0CI@LPOJHEHM@?$CK?5ProcessIoctl?3?5DBG_ISR_TRACE?5fl@FNODOBFM@ 0041f9f0     ioctl.obj
 0001:0001ea18       ??_C@_0DC@NOLFHCLF@?$CK?5ProcessIoctl?3?5DBG_IO_FUNC_ENTR@FNODOBFM@ 0041fa18     ioctl.obj
 0001:0001ea4a       ??_C@_0DE@PFEFFOBG@?$CK?5ProcessIoctl?3?5DBG_INIT_FUNC_EN@FNODOBFM@ 0041fa4a     ioctl.obj
 0001:0001ea7e       ??_C@_0DF@DPLBBPBM@?$CK?5ProcessIoctl?3?5DBG_IOCTL_FUNC_E@FNODOBFM@ 0041fa7e     ioctl.obj
 0001:0001eab4       ??_C@_0CL@GAIHEBC@?$CK?5ProcessIoctl?3?5DBG_IO_TRACE?5fla@FNODOBFM@ 0041fab4     ioctl.obj
 0001:0001eae0       ??_C@_0CO@NGOEBBKH@?$CK?5ProcessIoctl?3?5DBG_IOCTL_TRACE?5@FNODOBFM@ 0041fae0     ioctl.obj
 0001:0001eb0e       ??_C@_0DA@HPMIGAD@?$CK?5ProcessIoctl?3?5DBG_CLUSTER_TRAC@FNODOBFM@ 0041fb0e     ioctl.obj
 0001:0001eb3e       ??_C@_0CM@NECMPDIP@?$CK?5ProcessIoctl?3?5DBG_ISR_TRACE?5fl@FNODOBFM@ 0041fb3e     ioctl.obj
 0001:0001eb6a       ??_C@_0DG@PHFPGNCH@?$CK?5ProcessIoctl?3?5DBG_IO_FUNC_ENTR@FNODOBFM@ 0041fb6a     ioctl.obj
 0001:0001eba0       ??_C@_0DI@CBNGHMLF@?$CK?5ProcessIoctl?3?5DBG_INIT_FUNC_EN@FNODOBFM@ 0041fba0     ioctl.obj
 0001:0001ebd8       ??_C@_0DJ@DEFCHEDB@?$CK?5ProcessIoctl?3?5DBG_IOCTL_FUNC_E@FNODOBFM@ 0041fbd8     ioctl.obj
 0001:0001ec12       ??_C@_0CC@ELKJFKAD@?$CK?5ProcessIoctl?3?5DebugFlags?3?50x?$CFx@FNODOBFM@ 0041fc12     ioctl.obj
 0001:0001ec34       ??_C@_0DI@PNEPHAGL@?$CK?5Set?5pInitStruct?9?$DONoOfMsiVector@FNODOBFM@ 0041fc34     ioctl.obj
 0001:0001ec6c       ??_C@_0DF@KDDHBOCK@?$CK?5when?5back?5from?5IOP_RESET?0?5we?5w@FNODOBFM@ 0041fc6c     ioctl.obj
 0001:0001eca2       ??_C@_0DO@IBFHJCIJ@?$CK?5IOP?5RESET?5is?5done?5in?5ProcessIo@FNODOBFM@ 0041fca2     ioctl.obj
 0001:0001ece0       ??_C@_0DN@EJCEJBIF@?$CK?5IOP?5RESET?5failed?5in?5ProcessIoc@FNODOBFM@ 0041fce0     ioctl.obj
 0001:0001ed1e       ??_C@_0CF@GENCHGED@?$CK?5ProcessIoctl?3?5coalescing?5disab@FNODOBFM@ 0041fd1e     ioctl.obj
 0001:0001ed44       ??_C@_0CE@KOEFFOB@?$CK?5ProcessIoctl?3?5coalescing?5enabl@FNODOBFM@ 0041fd44     ioctl.obj
 0001:0001ed68       ??_C@_0GG@KLCLOEBM@?$CK?5ProcessIoctl?3?5Get?5a?5request?5fo@FNODOBFM@ 0041fd68     ioctl.obj
 0001:0001edce       ??_C@_0IA@OEPDMML@?$CK?5ProcessIoctl?3?5Get?5a?5request?5fo@FNODOBFM@ 0041fdce     ioctl.obj
 0001:0001ee4e       ??_C@_0GG@JMGDPGEE@?$CK?5ProcessIoctl?3?5Get?5a?5request?5fo@FNODOBFM@ 0041fe4e     ioctl.obj
 0001:0001eeb4       ??_C@_0IA@HMGAPIGO@?$CK?5ProcessIoctl?3?5Get?5a?5request?5fo@FNODOBFM@ 0041feb4     ioctl.obj
 0001:0001ef34       ??_C@_0DH@GFOJOHEG@?$CK?5ProcessIoctl?3?5TTYPE_CHANGE_IO_@FNODOBFM@ 0041ff34     ioctl.obj
 0001:0001ef6c       ??_C@_0CN@FFFLABJM@?$CK?5ProcessIoctl?3?5AIF?5commands?5pri@FNODOBFM@ 0041ff6c     ioctl.obj
 0001:0001ef9a       ??_C@_0CO@EKDJMEJG@?$CK?5ProcessIoctl?3?5AIF?5commands?5pri@FNODOBFM@ 0041ff9a     ioctl.obj
 0001:0001efc8       ??_C@_0CP@DNDOBHJJ@?$CK?5ProcessIoctl?3?5synch?5commands?5p@FNODOBFM@ 0041ffc8     ioctl.obj
 0001:0001eff8       ??_C@_0DA@DKDLFFAP@?$CK?5ProcessIoctl?3?5synch?5commands?5p@FNODOBFM@ 0041fff8     ioctl.obj
 0001:0001f028       ??_C@_0DD@OCMBIILM@?$CK?5ProcessIoctl?3?5RUN_CODE_IN_SPEC@FNODOBFM@ 00420028     ioctl.obj
 0001:0001f05c       ??_C@_0FD@PBJMMHDI@?$CK?5ProcessIoctl?3?5RUN_CODE_IN_SPEC@FNODOBFM@ 0042005c     ioctl.obj
 0001:0001f0b0       ??_C@_0EG@IJGFKELB@?$CK?5ProcessIoctl?3?5bus?$DN?$CFd?0?5target?$DN?$CF@FNODOBFM@ 004200b0     ioctl.obj
 0001:0001f0f6       ??_C@_0GB@LAAKBHJK@?$CK?5ProcessIoctl?3?5wrong?5parameters@FNODOBFM@ 004200f6     ioctl.obj
 0001:0001f158       ??_C@_0DD@LPBHEFLI@?$CK?5ProcessIoctl?3?5OsCmd?5?$CF2d?3?5cmd?$CI0@FNODOBFM@ 00420158     ioctl.obj
 0001:0001f18c       ??_C@_0DN@BFALKLFI@?$CK?5ProcessIoctl?3?5Osioctl?5?$CF2d?3?5con@FNODOBFM@ 0042018c     ioctl.obj
 0001:0001f1ca       ??_C@_0DA@LCPJHFEI@?$CK?5ProcessIoctl?3?5Max?5Data?5Transfe@FNODOBFM@ 004201ca     ioctl.obj
 0001:0001f1fa       ??_C@_0CE@DJCKDJAF@?$CK?5ProcessIoctl?3?5Max?5SG?5items?3?50x@FNODOBFM@ 004201fa     ioctl.obj
 0001:0001f21e       ??_C@_0BF@JHMLOOKE@?$CK?5outstanding?5IO?3?$CFd?6?$AA@FNODOBFM@ 0042021e     ioctl.obj
 0001:0001f234       ??_C@_0BO@MJJJDCNP@?$CK?5Coalescing?5Q?4?5CalledCnt?3?$CFd?6?$AA@FNODOBFM@ 00420234     ioctl.obj
 0001:0001f252       ??_C@_0CJ@GBKALEBA@?$CK?5Coalescing?5Q?4?5Beyond8kTransfer@FNODOBFM@ 00420252     ioctl.obj
 0001:0001f27c       ??_C@_0CJ@OEJKDMEF@?$CK?5Coalescing?5Q?4?5AcrossStripeBoun@FNODOBFM@ 0042027c     ioctl.obj
 0001:0001f2a6       ??_C@_0CD@JOOBICJM@?$CK?5Coalescing?5Q?4?5RwCmdTypeMixed?3?$CF@FNODOBFM@ 004202a6     ioctl.obj
 0001:0001f2ca       ??_C@_0CD@HLIMFKCF@?$CK?5Coalescing?5Q?4?5SGcntOverLimit?3?$CF@FNODOBFM@ 004202ca     ioctl.obj
 0001:0001f2ee       ??_C@_0CF@HPODEDGN@?$CK?5Coalescing?5Q?4?5CmdSizeOverLimit@FNODOBFM@ 004202ee     ioctl.obj
 0001:0001f314       ??_C@_0CF@HCLMLLN@?$CK?5Coalescing?5Q?4?5DequeueCalledCnt@FNODOBFM@ 00420314     ioctl.obj
 0001:0001f33a       ??_C@_0CL@HMCMDMGE@?$CK?5Coalescing?5Q?4?5CallSendFibDirec@FNODOBFM@ 0042033a     ioctl.obj
 0001:0001f366       ??_C@_0BL@BDGJNAIM@?$CK?5Sorting?5Q?4?5CalledCnt?3?$CFd?6?$AA@FNODOBFM@ 00420366     ioctl.obj
 0001:0001f382       ??_C@_0BO@FHMIKIJB@?$CK?5Sorting?5Q?4?5OverlapCase1?3?$CFd?6?$AA@FNODOBFM@ 00420382     ioctl.obj
 0001:0001f3a0       ??_C@_0BO@NBFMNKDP@?$CK?5Sorting?5Q?4?5OverlapCase2?3?$CFd?6?$AA@FNODOBFM@ 004203a0     ioctl.obj
 0001:0001f3be       ??_C@_0CK@EPAOGNLF@?$CK?5ProcessIoctl?3?5BUILDIO?5LOOPBACK@FNODOBFM@ 004203be     ioctl.obj
 0001:0001f3e8       ??_C@_0CK@DADBMBLL@?$CK?5ProcessIoctl?3?5STARTIO?5LOOPBACK@FNODOBFM@ 004203e8     ioctl.obj
 0001:0001f412       ??_C@_0CK@BMBGJMJA@?$CK?5ProcessIoctl?3?5PUSHFIB?5LOOPBACK@FNODOBFM@ 00420412     ioctl.obj
 0001:0001f43c       ??_C@_0CL@DANMEPHG@?$CK?5ProcessIoctl?3?5BUILDIO?5LOOPBACK@FNODOBFM@ 0042043c     ioctl.obj
 0001:0001f468       ??_C@_0CL@NHBLFNNN@?$CK?5ProcessIoctl?3?5STARTIO?5LOOPBACK@FNODOBFM@ 00420468     ioctl.obj
 0001:0001f494       ??_C@_0CL@HLILIDMA@?$CK?5ProcessIoctl?3?5PUSHFIB?5LOOPBACK@FNODOBFM@ 00420494     ioctl.obj
 0001:0001f4c0       ??_C@_0DB@MDNCKDFE@?$CK?5ProcessIoctl?3?5Simulate?5SCSI?5sm@FNODOBFM@ 004204c0     ioctl.obj
 0001:0001f4f2       ??_C@_0EC@KMBGJBEG@?$CK?5ProcessIoctl?3?5Simulate?5FW?5Targ@FNODOBFM@ 004204f2     ioctl.obj
 0001:0001f534       ??_C@_0BI@COAKNOP@?$CK?5?9?5IOCTL?5MESSAGE?3?5?$CFs?5?6?$AA@FNODOBFM@ 00420534     ioctl.obj
 0001:0001f54c       ??_C@_0BP@PHOOCPMJ@?$CK?5?9?5IOCTL?3?5FSAMPCTL_RESET_IOP?6?$AA@FNODOBFM@ 0042054c     ioctl.obj
 0001:0001f56c       ??_C@_0L@EIJBKGJP@arcsas?4sys?$AA@FNODOBFM@ 0042056c     ioctl.obj
 0001:0001f578       ??_C@_0BN@BIKJANKI@Adaptec?5RAID?5Storport?5Driver?$AA@FNODOBFM@ 00420578     ioctl.obj
 0001:0001f596       ??_C@_0DJ@MIENLJJJ@OMR?5value?5in?5Check?5Adapter?5Healt@FNODOBFM@ 00420596     comm.obj
 0001:0001f5d0       ??_C@_0CM@GEHGCFFI@?$CK?5ProcessAif?3?5AIF?5cmd?3?5?$CFd?0?5AIF?5s@FNODOBFM@ 004205d0     comm.obj
 0001:0001f5fc       ??_C@_1FE@JLJHJCGF@?$AAA?$AAr?$AAr?$AAa?$AAy?$AA?5?$AAm?$AAi?$AAg?$AAr?$AAa?$AAt?$AAi?$AAo?$AAn?$AA?1?$AAe?$AAx?$AAp?$AAa?$AAn?$AAs?$AAi?$AAo?$AAn?$AA?5?$AAc?$AAo?$AAm?$AAp?$AAl?$AAe@FNODOBFM@ 004205fc     comm.obj
 0001:0001f650       ??_C@_0CJ@ELNMEDDG@AIF?5EVENT?3?5Container?5?$CD?$CFd?5Morph?5c@FNODOBFM@ 00420650     comm.obj
 0001:0001f67a       ??_C@_1CK@DJNKNDAB@?$AAR?$AAa?$AAw?$AA?5?$AAD?$AAr?$AAi?$AAv?$AAe?$AA?5?$AAr?$AAe?$AAm?$AAo?$AAv?$AAe?$AAd?$AA?0?$AA?5?$AA?$CD?$AA?$AA@FNODOBFM@ 0042067a     comm.obj
 0001:0001f6a4       ??_C@_0CF@GOGNODAJ@AIF?5EVENT?3?5a?5RAW?5device?5?$CD?$CFd?5remo@FNODOBFM@ 004206a4     comm.obj
 0001:0001f6ca       ??_C@_1DG@JPPGPNNE@?$AAN?$AAa?$AAt?$AAi?$AAv?$AAe?$AA?5?$AAH?$AAB?$AAA?$AA?5?$AAd?$AAe?$AAv?$AAi?$AAc?$AAe?$AA?5?$AAi?$AAs?$AA?5?$AAa?$AAd?$AAd?$AAe?$AAd?$AA?$AA@FNODOBFM@ 004206ca     comm.obj
 0001:0001f700       ??_C@_0CL@PFPKJCEB@AIF?5EVENT?3?5AifEnNativeHBADeviceA@FNODOBFM@ 00420700     comm.obj
 0001:0001f72c       ??_C@_1DK@DMPEAPAK@?$AAN?$AAa?$AAt?$AAi?$AAv?$AAe?$AA?5?$AAH?$AAB?$AAA?$AA?5?$AAd?$AAe?$AAv?$AAi?$AAc?$AAe?$AA?5?$AAi?$AAs?$AA?5?$AAr?$AAe?$AAm?$AAo?$AAv?$AAe?$AAd?$AA?$AA@FNODOBFM@ 0042072c     comm.obj
 0001:0001f766       ??_C@_0CO@KNHKMPNF@AIF?5EVENT?3?5AifEnNativeHBADeviceR@FNODOBFM@ 00420766     comm.obj
 0001:0001f794       ??_C@_1EO@PNKAKFGH@?$AAH?$AAa?$AAr?$AAd?$AAw?$AAa?$AAr?$AAe?$AA?5?$AAn?$AAo?$AAt?$AA?5?$AAp?$AAr?$AAe?$AAs?$AAe?$AAn?$AAt?$AA?9?$AA?5?$AAB?$AAa?$AAc?$AAk?$AAu?$AAp?$AA?5?$AAn?$AAo?$AAt@FNODOBFM@ 00420794     comm.obj
 0001:0001f7e2       ??_C@_0DD@GCBHPPGK@AIF?5EVENT?3?5Hardware?5not?5present?9@FNODOBFM@ 004207e2     comm.obj
 0001:0001f816       ??_C@_1CI@IELPCEHF@?$AAS?$AAu?$AAp?$AAe?$AAr?$AAc?$AAa?$AAp?$AA?5?$AAh?$AAe?$AAa?$AAl?$AAt?$AAh?$AA?5?$AAl?$AAo?$AAw?$AA?$AA@FNODOBFM@ 00420816     comm.obj
 0001:0001f83e       ??_C@_0EJ@OLDMFEFC@AIF?5EVENT?3?5Super?5cap?5health?5is?5l@FNODOBFM@ 0042083e     comm.obj
 0001:0001f888       ??_C@_1CK@BAADJOPA@?$AAS?$AAu?$AAp?$AAe?$AAr?$AAc?$AAa?$AAp?$AA?5?$AAh?$AAe?$AAa?$AAl?$AAt?$AAh?$AA?5?$AA?5?$AAb?$AAa?$AAd?$AA?$AA@FNODOBFM@ 00420888     comm.obj
 0001:0001f8b2       ??_C@_0DM@BNKBKMII@AIF?5EVENT?3?5Super?5cap?5health?5is?5b@FNODOBFM@ 004208b2     comm.obj
 0001:0001f8ee       ??_C@_1CA@DNJAAJKJ@?$AAC?$AAa?$AAc?$AAh?$AAe?$AA?5?$AAd?$AAa?$AAt?$AAa?$AA?5?$AAl?$AAo?$AAs?$AAs?$AA?$AA@FNODOBFM@ 004208ee     comm.obj
 0001:0001f90e       ??_C@_0BM@DGCCGGOI@AIF?5EVENT?3?5Cache?5data?5loss?6?$AA@FNODOBFM@ 0042090e     comm.obj
 0001:0001f92a       ??_C@_1DG@KILEJPC@?$AAT?$AAe?$AAm?$AAp?$AAe?$AAr?$AAa?$AAt?$AAu?$AAr?$AAe?$AA?5?$AAB?$AAa?$AAc?$AAk?$AA?5?$AAt?$AAo?$AA?5?$AAN?$AAo?$AAr?$AAm?$AAa?$AAl?$AA?$AA@FNODOBFM@ 0042092a     comm.obj
 0001:0001f960       ??_C@_0CH@EOEMJJE@AIF?5EVENT?3?5Temperature?5Back?5to?5N@FNODOBFM@ 00420960     comm.obj
 0001:0001f988       ??_C@_1DG@IHOODPDN@?$AAS?$AAu?$AAp?$AAe?$AAr?$AAc?$AAa?$AAp?$AA?5?$AAT?$AAe?$AAm?$AAp?$AAe?$AAr?$AAa?$AAt?$AAu?$AAr?$AAe?$AA?5?$AAA?$AAl?$AAe?$AAr?$AAt?$AA?$AA@FNODOBFM@ 00420988     comm.obj
 0001:0001f9be       ??_C@_0EA@EGACBNC@AIF?5EVENT?3?5Temperature?5has?5cross@FNODOBFM@ 004209be     comm.obj
 0001:0001f9fe       ??_C@_1DK@KKLIINGO@?$AAS?$AAu?$AAp?$AAe?$AAr?$AAc?$AAa?$AAp?$AA?5?$AAT?$AAe?$AAm?$AAp?$AAe?$AAr?$AAa?$AAt?$AAu?$AAr?$AAe?$AA?5?$AAW?$AAa?$AAr?$AAn?$AAi?$AAn?$AAg?$AA?$AA@FNODOBFM@ 004209fe     comm.obj
 0001:0001fa38       ??_C@_0ED@CGHEBKG@AIF?5EVENT?3?5Temperature?5is?5in?5the@FNODOBFM@ 00420a38     comm.obj
 0001:0001fa7c       ??_C@_1DK@HENHBAOO@?$AAB?$AAa?$AAc?$AAk?$AAu?$AAp?$AA?5?$AAu?$AAn?$AAi?$AAt?$AA?5?$AAs?$AAe?$AAl?$AAf?$AA?9?$AAt?$AAe?$AAs?$AAt?$AA?5?$AAf?$AAa?$AAi?$AAl?$AAe?$AAd?$AA?$AA@FNODOBFM@ 00420a7c     comm.obj
 0001:0001fab6       ??_C@_0CJ@JLLJHFCM@AIF?5EVENT?3?5Backup?5unit?5self?9test@FNODOBFM@ 00420ab6     comm.obj
 0001:0001fae0       ??_C@_1DK@GKIHJFEC@?$AAF?$AAa?$AAt?$AAa?$AAl?$AA?5?$AAE?$AAr?$AAr?$AAo?$AAr?$AA?3?$AA?5?$AAB?$AAa?$AAc?$AAk?$AAu?$AAp?$AA?5?$AAd?$AAi?$AAs?$AAa?$AAb?$AAl?$AAe?$AAd?$AA?$AA@FNODOBFM@ 00420ae0     comm.obj
 0001:0001fb1a       ??_C@_0CJ@NHDLILDM@AIF?5EVENT?3?5Fatal?5Error?3?5Backup?5d@FNODOBFM@ 00420b1a     comm.obj
 0001:0001fb44       ??_C@_1CO@DFMHCOAI@?$AAL?$AAo?$AAg?$AAi?$AAc?$AAa?$AAl?$AA?5?$AAD?$AAr?$AAi?$AAv?$AAe?$AA?5?$AAa?$AAd?$AAd?$AAe?$AAd?$AA?0?$AA?5?$AA?$CD?$AA?$AA@FNODOBFM@ 00420b44     comm.obj
 0001:0001fb72       ??_C@_0CA@GLOIGEIG@AIF?5EVENT?3?5Container?5?$CD?$CFd?5added?6?$AA@FNODOBFM@ 00420b72     comm.obj
 0001:0001fb92       ??_C@_1DC@CMPCKFLI@?$AAL?$AAo?$AAg?$AAi?$AAc?$AAa?$AAl?$AA?5?$AAD?$AAr?$AAi?$AAv?$AAe?$AA?5?$AAd?$AAe?$AAl?$AAe?$AAt?$AAe?$AAd?$AA?0?$AA?5?$AA?$CD?$AA?$AA@FNODOBFM@ 00420b92     comm.obj
 0001:0001fbc4       ??_C@_0CC@IGLGEBDK@AIF?5EVENT?3?5Container?5?$CD?$CFd?5removed@FNODOBFM@ 00420bc4     comm.obj
 0001:0001fbe6       ??_C@_0FE@GFLJPFDG@AIF?5EVENT?3?5AifEnEnclosureManagem@FNODOBFM@ 00420be6     comm.obj
 0001:0001fc3a       ??_C@_1CI@JDGBIDGK@?$AAA?$AA?5?$AAn?$AAe?$AAw?$AA?5?$AAJ?$AAB?$AAO?$AAD?$AA?5?$AAi?$AAs?$AA?5?$AAa?$AAd?$AAd?$AAe?$AAd?$AA?$AA@FNODOBFM@ 00420c3a     comm.obj
 0001:0001fc62       ??_C@_0BJ@NJMLAEMO@AIF?5EVENT?3?5a?5JBOD?5added?6?$AA@FNODOBFM@ 00420c62     comm.obj
 0001:0001fc7c       ??_C@_1CE@CICPDMOD@?$AAA?$AA?5?$AAJ?$AAB?$AAO?$AAD?$AA?5?$AAi?$AAs?$AA?5?$AAd?$AAe?$AAl?$AAe?$AAt?$AAe?$AAd?$AA?$AA@FNODOBFM@ 00420c7c     comm.obj
 0001:0001fca0       ??_C@_0BL@PDKEFHEM@AIF?5EVENT?3?5a?5JBOD?5removed?6?$AA@FNODOBFM@ 00420ca0     comm.obj
 0001:0001fcbc       ??_C@_0DO@DNJOKEFB@AIF?5EVENT?3?5AifCmdJobProgress?5for@FNODOBFM@ 00420cbc     comm.obj
 0001:0001fcfa       ??_C@_0EM@MHLKFBIP@AIF?5EVENT?3?5AifCmdJobProgress?5for@FNODOBFM@ 00420cfa     comm.obj
 0001:0001fd46       ??_C@_0CG@IPLFJLPL@Smart?5HBA?5Scsi?5response?5Status?5?$DN@FNODOBFM@ 00420d46     comm.obj
 0001:0001fd6c       ??_C@_0DO@HNDDHFGA@?5HBA?5Error?5HBA_MODE_DISABLED?5Srb@FNODOBFM@ 00420d6c     comm.obj
 0001:0001fdaa       ??_C@_0DA@CPGPCCBA@?5HBA?5Error?5code?5?$CFx?5For?5Path?5ID?5?$CF@FNODOBFM@ 00420daa     comm.obj
 0001:0001fdda       ??_C@_0FA@CPHJLELC@?5HBA?5Error?5SCSI_COMPL_TRANSL_STA@FNODOBFM@ 00420dda     comm.obj
 0001:0001fe2a       ??_C@_0FE@JFIIIBKF@?5HBA?5Error?5SCSI_COMPL_TRANSL_STA@FNODOBFM@ 00420e2a     comm.obj
 0001:0001fe7e       ??_C@_0EO@DHIENLOG@?5HBA?5Error?3?5Length?5from?5OS?$CI0x?$CFx?$CJ@FNODOBFM@ 00420e7e     comm.obj
 0001:0001fecc       ??_C@_0HP@ECKDIFKN@?5HBA?5Error?3?5hbaCmd?9?$DOdata_length?$CI@FNODOBFM@ 00420ecc     comm.obj
 0001:0001ff4c       ??_C@_0FK@IBAGLEPN@?5HBA?5Error?5SCSI_COMPL_TRANSL_STA@FNODOBFM@ 00420f4c     comm.obj
 0001:0001ffa6       ??_C@_0FJ@DMCDLFNM@?5HBA?5Error?5SCSI_COMPL_TRANSL_STA@FNODOBFM@ 00420fa6     comm.obj
 0001:00020000       ??_C@_0EP@JHLDIODO@?$CK?5NO?5ERROR?5handling?5for?5pHbaResp@FNODOBFM@ 00421000     comm.obj
 0001:00020050       ??_C@_0CG@PJJANG@TMF?5Function?5Completed?5Successfu@FNODOBFM@ 00421050     comm.obj
 0001:00020076       ??_C@_0FJ@OIALMBME@?$CK?5NO?5ERROR?5handling?5for?5pHbaResp@FNODOBFM@ 00421076     comm.obj
 0001:000200d0       ??_C@_1BI@BHAHBMFJ@?$AAM?$AAo?$AAf?$AAR?$AAe?$AAs?$AAo?$AAu?$AAr?$AAc?$AAe?$AA?$AA@FNODOBFM@ 004210d0     wmi.obj
 0001:000200e8       ??_C@_1BK@EPHGJNJ@?$AAS?$AAc?$AAs?$AAi?$AAM?$AAi?$AAn?$AAi?$AAP?$AAo?$AAr?$AAt?$AA?$AA@FNODOBFM@ 004210e8     scsiwmi:wmilib.obj
 0002:00000000       __imp___aulldvrm           00422000     ntoskrnl:ntoskrnl.exe
 0002:00000004       __imp___alldiv             00422004     ntoskrnl:ntoskrnl.exe
 0002:00000008       __imp___allmul             00422008     ntoskrnl:ntoskrnl.exe
 0002:0000000c       __imp___aulldiv            0042200c     ntoskrnl:ntoskrnl.exe
 0002:00000010       __imp___aullshr            00422010     ntoskrnl:ntoskrnl.exe
 0002:00000014       __imp__memset              00422014     ntoskrnl:ntoskrnl.exe
 0002:00000018       \177ntoskrnl_NULL_THUNK_DATA 00422018     ntoskrnl:ntoskrnl.exe
 0002:0000001c       __imp__StorPortGetPhysicalAddress@16 0042201c     storport:storport.sys
 0002:00000020       __imp__StorPortResumeDevice@16 00422020     storport:storport.sys
 0002:00000024       __imp__StorPortNotification 00422024     storport:storport.sys
 0002:00000028       __imp__StorPortStallExecution@4 00422028     storport:storport.sys
 0002:0000002c       __imp__StorPortReadRegisterUchar@8 0042202c     storport:storport.sys
 0002:00000030       __imp__StorPortReadRegisterUlong@8 00422030     storport:storport.sys
 0002:00000034       __imp__StorPortReadRegisterBufferUchar@16 00422034     storport:storport.sys
 0002:00000038       __imp__StorPortWriteRegisterUlong@12 00422038     storport:storport.sys
 0002:0000003c       __imp__StorPortWriteRegisterBufferUlong@16 0042203c     storport:storport.sys
 0002:00000040       __imp__StorPortMoveMemory@12 00422040     storport:storport.sys
 0002:00000044       __imp__StorPortDebugPrint  00422044     storport:storport.sys
 0002:00000048       __imp__StorPortGetDeviceBase@28 00422048     storport:storport.sys
 0002:0000004c       __imp__StorPortWriteRegisterBufferUchar@16 0042204c     storport:storport.sys
 0002:00000050       __imp__StorPortResume@4    00422050     storport:storport.sys
 0002:00000054       __imp__StorPortInitialize@16 00422054     storport:storport.sys
 0002:00000058       __imp__StorPortFreeDeviceBase@8 00422058     storport:storport.sys
 0002:0000005c       __imp__StorPortGetBusData@24 0042205c     storport:storport.sys
 0002:00000060       __imp__StorPortGetUncachedExtension@12 00422060     storport:storport.sys
 0002:00000064       __imp__StorPortPause@8     00422064     storport:storport.sys
 0002:00000068       __imp__StorPortSetDeviceQueueDepth@20 00422068     storport:storport.sys
 0002:0000006c       __imp__StorPortQuerySystemTime@4 0042206c     storport:storport.sys
 0002:00000070       __imp__StorPortExtendedFunction 00422070     storport:storport.sys
 0002:00000074       __imp__StorPortPauseDevice@20 00422074     storport:storport.sys
 0002:00000078       __imp__StorPortBusy@8      00422078     storport:storport.sys
 0002:0000007c       __imp__StorPortGetScatterGatherList@8 0042207c     storport:storport.sys
 0002:00000080       __imp__ScsiPortMoveMemory@12 00422080     storport:storport.sys
 0002:00000084       \177storport_NULL_THUNK_DATA 00422084     storport:storport.sys
 0002:00000128       _RevCompareTable           00422128     revision.obj
 0002:00000228       _RevCompareTableLength     00422228     revision.obj
 0002:000002ec       ??_C@_08HNOCAICB@Adaptec?5?$AA@ 004222ec     arcsas.obj
 0002:000002f8       ??_C@_04ODJNANJC@9005?$AA@ 004222f8     arcsas.obj
 0002:00000300       ??_C@_04EKJHPGNA@0285?$AA@ 00422300     arcsas.obj
 0002:00000308       ??_C@_04GBLKKFBD@0286?$AA@ 00422308     arcsas.obj
 0002:00000310       ??_C@_04PPDJIIJN@0288?$AA@ 00422310     arcsas.obj
 0002:00000318       ??_C@_04LPGNDNED@028b?$AA@ 00422318     arcsas.obj
 0002:00000320       ??_C@_04KGHGAMAC@028c?$AA@ 00422320     arcsas.obj
 0002:00000328       ??_C@_04OJDHJKMF@028d?$AA@ 00422328     arcsas.obj
 0002:00000330       ??_C@_0BB@MMDKHCIH@ARC?9SAS?5?5?5?5?5?5?5?5?5?$AA@ 00422330     arcsas.obj
 0002:00000344       ??_C@_06DFBHEALI@AACAPI?$AA@ 00422344     arcsas.obj
 0002:00000470       __load_config_used         00422470     BufferOverflowFastFailK:loadcfg.obj
 0002:00000500       ___safe_se_handler_table   00422500     <linker-defined>
 0003:00000000       _gDebugFlags               00423000     arcdebug.obj
 0003:00000008       _gNativeModeAdapters       00423008     arcsas.obj
 0003:000001b8       _gNumNativeModeAdapters    004231b8     arcsas.obj
 0003:000001bc       _gARCProductId             004231bc     arcsas.obj
 0003:000001c0       _gARCApiId                 004231c0     arcsas.obj
 0003:000001c4       _gARCOEMFlags              004231c4     arcsas.obj
 0003:000001c8       _gARCSASRxSubsystemInfo    004231c8     arcsas.obj
 0003:00000350       _gARCSASRktSubsystemInfo   00423350     arcsas.obj
 0003:00000388       _gARCSASArkSubsystemInfo   00423388     arcsas.obj
 0003:000003a0       _gARCSASPMCSubsystemInfo   004233a0     arcsas.obj
 0003:000004a0       _gARCVendor                004234a0     arcinit.obj
 0003:000004a4       _gAdapterGuid              004234a4     wmi.obj
 0003:000004b4       _gIoChannelGuid            004234b4     wmi.obj
 0003:000004c4       _gDiskArrayGuid            004234c4     wmi.obj
 0003:000004d4       _gPhysicalDiskGuid         004234d4     wmi.obj
 0003:000004e4       _gAdapterMethodGuid        004234e4     wmi.obj
 0003:000004f4       ___security_cookie         004234f4     BufferOverflowFastFailK:gs_support.obj
 0003:000004f8       ___security_cookie_complement 004234f8     BufferOverflowFastFailK:gs_support.obj
 0003:00000520       _gTraceContext             00423520     arcinit.obj
 0003:00000524       _gAdapterAddCount          00423524     arcinit.obj
 0003:000005c0       _gAdapterTable             004235c0     <common>
 0003:000006c0       _gDriverObject             004236c0     <common>
 0004:00000006       ___security_init_cookie    00424006 f   BufferOverflowFastFailK:gs_support.obj
 0004:00000030       __IMPORT_DESCRIPTOR_ntoskrnl 00424030     ntoskrnl:ntoskrnl.exe
 0004:00000044       __IMPORT_DESCRIPTOR_storport 00424044     storport:storport.sys
 0004:00000058       __NULL_IMPORT_DESCRIPTOR   00424058     ntoskrnl:ntoskrnl.exe

 entry point at        0001:000188d0

 Static symbols

 0000:fffd8000       .debug$S                   00400000     storport:storport.sys
 0000:fffd8000       .debug$S                   00400000     storport:storport.sys
 0000:fffd8000       .debug$S                   00400000     storport:storport.sys
 0000:fffd8000       .debug$S                   00400000     storport:storport.sys
 0000:fffd8000       .debug$S                   00400000     storport:storport.sys
 0000:fffd8000       .debug$S                   00400000     storport:storport.sys
 0000:fffd8000       .debug$S                   00400000     storport:storport.sys
 0000:fffd8000       .debug$S                   00400000     storport:storport.sys
 0000:fffd8000       .debug$S                   00400000     storport:storport.sys
 0000:fffd8000       .debug$S                   00400000     storport:storport.sys
 0000:fffd8000       .debug$S                   00400000     storport:storport.sys
 0000:fffd8000       .debug$S                   00400000     storport:storport.sys
 0000:fffd8000       .debug$S                   00400000     storport:storport.sys
 0000:fffd8000       .debug$S                   00400000     ntoskrnl:ntoskrnl.exe
 0000:fffd8000       .debug$S                   00400000     ntoskrnl:ntoskrnl.exe
 0000:fffd8000       .debug$S                   00400000     ntoskrnl:ntoskrnl.exe
 0000:fffd8000       .debug$S                   00400000     ntoskrnl:ntoskrnl.exe
 0000:fffd8000       .debug$S                   00400000     ntoskrnl:ntoskrnl.exe
 0000:fffd8000       .debug$S                   00400000     ntoskrnl:ntoskrnl.exe
 0000:fffd8000       .debug$S                   00400000     storport:storport.sys
 0000:fffd8000       .debug$S                   00400000     storport:storport.sys
 0000:fffd8000       .debug$S                   00400000     storport:storport.sys
 0000:fffd8000       .debug$S                   00400000     storport:storport.sys
 0000:fffd8000       .debug$S                   00400000     storport:storport.sys
 0000:fffd8000       .debug$S                   00400000     storport:storport.sys
 0000:fffd8000       .debug$S                   00400000     storport:storport.sys
 0000:fffd8000       .debug$S                   00400000     storport:storport.sys
 0000:fffd8000       .debug$S                   00400000     storport:storport.sys
 0000:fffd8000       .debug$S                   00400000     storport:storport.sys
 0000:fffd8000       .debug$S                   00400000     storport:storport.sys
 0000:fffd8000       .debug$S                   00400000     storport:storport.sys
 0000:fffd8000       .debug$S                   00400000     storport:storport.sys
 0000:fffd8000       .debug$S                   00400000     storport:storport.sys
 0001:00001b10       $LN19                      00402b10     rxdevice.obj
 0001:00004658       $LN145                     00405658     arcdebug.obj
 0001:00004670       $LN138                     00405670     arcdebug.obj
 0001:000046a0       _StrcatLocal@8             004056a0 f   arcdebug.obj
 0001:000046e0       _Strcatc@8                 004056e0 f   arcdebug.obj
 0001:0000c140       $LN39                      0040d140     arcinit.obj
 0001:0000c370       $LN43                      0040d370     arcinit.obj
 0001:0000ccdc       $LN95                      0040dcdc     arcinit.obj
 0001:0000e958       $LN149                     0040f958     cmddelivery.obj
 0001:0000e980       $LN132                     0040f980     cmddelivery.obj
 0001:0000ea1c       $LN150                     0040fa1c     cmddelivery.obj
 0001:0000ea40       $LN133                     0040fa40     cmddelivery.obj
 0001:000105e8       $LN163                     004115e8     cmddelivery.obj
 0001:00010600       $LN150                     00411600     cmddelivery.obj
 0001:00010ca0       $LN43                      00411ca0     cmdproc.obj
 0001:00011acc       $LN160                     00412acc     cmdproc.obj
 0001:00011ae4       $LN147                     00412ae4     cmdproc.obj
 0001:00011b0c       $LN161                     00412b0c     cmdproc.obj
 0001:00011b1c       $LN148                     00412b1c     cmdproc.obj
 0001:00013abc       $LN24                      00414abc     ioctl.obj
 0001:00013aec       $LN19                      00414aec     ioctl.obj
 0001:00015eb4       $LN362                     00416eb4     ioctl.obj
 0001:00015ef4       $LN327                     00416ef4     ioctl.obj
 0001:00015f38       $LN363                     00416f38     ioctl.obj
 0001:00015f4c       $LN328                     00416f4c     ioctl.obj
 0001:00016d68       $LN91                      00417d68     comm.obj
 0001:00016d80       $LN92                      00417d80     comm.obj
 0001:00016da0       $LN71                      00417da0     comm.obj
 0001:00016dc8       $LN93                      00417dc8     comm.obj
 0001:000171b4       $LN35                      004181b4     comm.obj
 0001:000171d0       $LN32                      004181d0     comm.obj
 0001:00017ad4       $LN180                     00418ad4     comm.obj
 0001:00017ae8       $LN161                     00418ae8     comm.obj
 0001:00018d32       $LN81                      00419d32     scsiwmi:wmilib.obj
 0001:00018f78       $$000000                   00419f78     BufferOverflowFastFailK:forceseh.obj
 0002:000000c8       _STORPORT_POFX_ADAPTER_GUID 004220c8     rxdevice.obj
 0002:000000d8       _STORPORT_POFX_LUN_GUID    004220d8     rxdevice.obj
 0002:000000e8       _STORPORT_DEVICEOPERATION_SECURE_REPROVISION_GUID 004220e8     rxdevice.obj
 0002:000000f8       _STORPORT_POFX_ADAPTER_GUID 004220f8     revision.obj
 0002:00000108       _STORPORT_POFX_LUN_GUID    00422108     revision.obj
 0002:00000118       _STORPORT_DEVICEOPERATION_SECURE_REPROVISION_GUID 00422118     revision.obj
 0002:0000022c       _STORPORT_POFX_ADAPTER_GUID 0042222c     helpers.obj
 0002:0000023c       _STORPORT_POFX_LUN_GUID    0042223c     helpers.obj
 0002:0000024c       _STORPORT_DEVICEOPERATION_SECURE_REPROVISION_GUID 0042224c     helpers.obj
 0002:0000025c       _STORPORT_POFX_ADAPTER_GUID 0042225c     arcdebug.obj
 0002:0000026c       _STORPORT_POFX_LUN_GUID    0042226c     arcdebug.obj
 0002:0000027c       _STORPORT_DEVICEOPERATION_SECURE_REPROVISION_GUID 0042227c     arcdebug.obj
 0002:0000028c       _STORPORT_POFX_ADAPTER_GUID 0042228c     timer.obj
 0002:0000029c       _STORPORT_POFX_LUN_GUID    0042229c     timer.obj
 0002:000002ac       _STORPORT_DEVICEOPERATION_SECURE_REPROVISION_GUID 004222ac     timer.obj
 0002:000002bc       _STORPORT_POFX_ADAPTER_GUID 004222bc     arcsas.obj
 0002:000002cc       _STORPORT_POFX_LUN_GUID    004222cc     arcsas.obj
 0002:000002dc       _STORPORT_DEVICEOPERATION_SECURE_REPROVISION_GUID 004222dc     arcsas.obj
 0002:0000034c       _STORPORT_POFX_ADAPTER_GUID 0042234c     arcinit.obj
 0002:0000035c       _STORPORT_POFX_LUN_GUID    0042235c     arcinit.obj
 0002:0000036c       _STORPORT_DEVICEOPERATION_SECURE_REPROVISION_GUID 0042236c     arcinit.obj
 0002:0000037c       _STORPORT_POFX_ADAPTER_GUID 0042237c     cmddelivery.obj
 0002:0000038c       _STORPORT_POFX_LUN_GUID    0042238c     cmddelivery.obj
 0002:0000039c       _STORPORT_DEVICEOPERATION_SECURE_REPROVISION_GUID 0042239c     cmddelivery.obj
 0002:000003ac       _STORPORT_POFX_ADAPTER_GUID 004223ac     cmdproc.obj
 0002:000003bc       _STORPORT_POFX_LUN_GUID    004223bc     cmdproc.obj
 0002:000003cc       _STORPORT_DEVICEOPERATION_SECURE_REPROVISION_GUID 004223cc     cmdproc.obj
 0002:000003dc       _STORPORT_POFX_ADAPTER_GUID 004223dc     ioctl.obj
 0002:000003ec       _STORPORT_POFX_LUN_GUID    004223ec     ioctl.obj
 0002:000003fc       _STORPORT_DEVICEOPERATION_SECURE_REPROVISION_GUID 004223fc     ioctl.obj
 0002:0000040c       _STORPORT_POFX_ADAPTER_GUID 0042240c     comm.obj
 0002:0000041c       _STORPORT_POFX_LUN_GUID    0042241c     comm.obj
 0002:0000042c       _STORPORT_DEVICEOPERATION_SECURE_REPROVISION_GUID 0042242c     comm.obj
 0002:0000043c       _STORPORT_POFX_ADAPTER_GUID 0042243c     wmi.obj
 0002:0000044c       _STORPORT_POFX_LUN_GUID    0042244c     wmi.obj
 0002:0000045c       _STORPORT_DEVICEOPERATION_SECURE_REPROVISION_GUID 0042245c     wmi.obj
 0003:00000004       ?NeedToReadStatus@?1??CheckingFWAfterPowerStateChange@@9@9 00423004     timer.obj
 0003:00000005       ?NeedToCheckMSIX@?1??CheckingFWAfterPowerStateChange@@9@9 00423005     timer.obj
 0003:00000500       ?CurrentCmdCode@?1??RxSendSynchCommand@@9@9 00423500     rxdevice.obj
 0003:00000504       ?CalledCnt@?1??CheckFWPulseInCrashDumpMode@@9@9 00423504     timer.obj
 0003:00000508       ?TimerAge@?1??CheckingFWAfterPowerStateChange@@9@9 00423508     timer.obj
 0003:0000050c       ?DelayCnt4DualFWFlushSoftReset@?1??CheckingFWAfterPowerStateChange@@9@9 0042350c     timer.obj
 0003:00000510       ?pSavedDevExt@?1??CheckingFWAfterPowerStateChange@@9@9 00423510     timer.obj
 0003:00000514       ?TimerAge@?1??Reset_IOP_CompletionTimer@@9@9 00423514     timer.obj
 0003:00000518       ?status@?1??CheckingFWAfterPowerStateChange@@9@9 00423518     timer.obj
 0003:00000528       ?NewScanStarted@?1??ConfigureContainersRuntime@@9@9 00423528     arcinit.obj
 0003:00000529       ?LoopCount@?1??ConfigureContainersRuntime@@9@9 00423529     arcinit.obj
 0003:0000052a       ?busChange@?1??ConfigureContainersRuntime@@9@9 0042352a     arcinit.obj
 0003:0000052b       ?initialized@?1??DriverEntry@@9@9 0042352b     arcinit.obj
 0003:0000052c       ?containerCount@?1??ConfigureContainersRuntime@@9@9 0042352c     arcinit.obj
 0003:00000530       ?pSavedDevExt@?1??ConfigureContainersRuntime@@9@9 00423530     arcinit.obj
 0003:00000534       ?SkipSecondSynchCmd@?1??ConfigureContainersRuntime@@9@9 00423534     arcinit.obj
 0003:00000538       ?diskInfoResponse@?1??ConfigureContainersRuntime@@9@9 00423538     arcinit.obj
 0003:000005a0       ?ShutdownSent@?1??BuildIo@@9@9 004235a0     cmdproc.obj
 0004:00000136       .idata$6                   00424136     ntoskrnl:ntoskrnl.exe
 0004:000003d2       .idata$6                   004243d2     storport:storport.sys
 0005:000000d0       $R000000                   004250d0     arcsas.res
 0005:00000438       $R000368                   00425438     arcsas.res
